:1000000091C20000ACC20000ABC20000A8C2000058
:10001000A6C20000A4C20000A2C20000A0C200004C
:100020009EC200009CC2000068C6000098C200008A
:1000300096C2000094C2000092C2000090C200006C
:100040008EC200008CC200008AC2000088C200007C
:1000500086C2000084C2000082C2000080C200008C
:100060007EC200007CC200007AC2000078C200009C
:1000700076C2000074C2000072C2000070C20000AC
:100080006EC200006CC200006AC2000068C20000BC
:1000900066C2000064C2000062C2000060C20000CC
:1000A0005EC200005CC200005AC2000001430000B2
:1000B0005A0000005A014200000000000000014503
:1000C000455A5A5A5A5A5A0144000000000000008A
:1000D000014D000001FFFFFFFF014F00FFFF030084
:1000E0000000140342006C006900730073002D00CF
:1000F00042006F007800000004030904090229008F
:10010000010100E06409040000020300000009216D
:100110001101000122BD030705810340000107050D
:10012000020320000105010905A101850105091946
:1001300001291815002501750195188102A10005F6
:100140000109300931093209330934093509360901
:1001500037150026FF00350046FF00750895088119
:1001600002C005012507463B017504950165140988
:10017000398142650095018101750895018103056A
:100180000F0992A1028502099415002501750895B1
:10019000018102750895018103C00921A102850131
:1001A0000922150125283501452875089501910278
:1001B0000925A10209260927093009310932093325
:1001C000093409400941250715013501450775081E
:1001D00095019100C009500954095175109503917A
:1001E0000255006600000952150026FF0035004642
:1001F0001027750895019102095375089501910220
:100200000955A102050109300931750195029102D4
:10021000C0050F095695019102950591030957A153
:10022000020B01000A000B02000A007508950291FA
:1002300002C0050F09A7751095019102C0050F09AD
:100240005AA10285020922750895019102095B09EC
:100250005D95029102095C095E75109102C0095F0B
:10026000A1028503092215012528350145287508B5
:1002700095019102092315002501350045017504FA
:10028000950191020958A1020B01000A000B02001E
:100290000A00750295029102C01580257F096075DC
:1002A00008950191020961096295029102150026E3
:1002B000FF000963096475089502910209659501BB
:1002C0009102C0096EA10285040922150125283575
:1002D0000145287508950191020970150026FF0057
:1002E0003500461027750895019102096F15802584
:1002F0007F36F0D8461027950191020971661400E7
:1003000055FE910209727510950191026600005523
:1003100000C00973A10285050922150125283501B0
:10032000452875089501910209701601FF26FF0006
:1003300036F0D8461027751095019102C00974A1B6
:1003400002850609221501252875089501910209E3
:100350007509761580257F750895029102C0050FF5
:100360000977A102850A09221501252835014528AA
:100370007508950191020978A1020979097A097B2A
:1003800015012503750895019100C0097C1500260B
:10039000FF00350046FF009102C00990A102850BC5
:1003A0000922750895019102C00996A102850C09E0
:1003B0009709980999099A099B099C1501250675C1
:1003C0000895019100C0097DA102850D097E75087F
:1003D00095019102C009ABA102850F0925A102096F
:1003E000260927093009310932093309340940093E
:1003F00041250715013501450775089501B100C074
:100400000501093B150026FF01350046FF01750A6D
:100410009501B1027506B101C0050F0989A10285D8
:10042000020922252815013501452875089501B1D5
:1004300002098BA102098C098D098E25031501354E
:1004400001450375089501B100C009AC751095010F
:10045000B100C0097FA1028503098075109501B123
:1004600002098375089501B10209A909AA750195C8
:1004700002B10275069501B103C00901A101150081
:1004800026FF0075088510950D0900B2020185113F
:1004900095050900B202018515950D0900B202010A
:1004A00085169600010900B20201851795300900F2
:1004B000B20201851995810900B2020185129508E1
:1004C0000900B202018513951C0900B202018518CA
:1004D00095C00900B20201851495C40900B2020159
:1004E000C0C00902300001010080FA0904000002C6
:1004F000FF5D01001021100101248114030003138A
:1005000002000300070581034000040705020340C1
:10051000000812010002FFFFFF405E048E0201018D
:100520000102030111241FBECFEFDAE0DEBFCDBF11
:1005300012E0A0E0B1E0ECE6F4E702C005900D9215
:10054000AA3FB107D9F726E0AAEFB2E001C01D9299
:10055000AD3BB207E1F70E94E12F0C94343A50CD45
:1005600090E090933D000F920FB60F922F933F9320
:100570004F93AF93BF935F93A4E6B5E0409115030B
:10058000221B38E09FE29A95F1F720E04899286015
:100590009AE09A95F1F7489B57C04999226000006C
:1005A0000000000092E09A95F1F7489921609EEBD7
:1005B0009A95F1F74999FECF0000413021F00000F3
:1005C0000000303001F0000000000000499908945C
:1005D0002D932227221F92E09A95F1F748990894CB
:1005E000221F93E09A95F1F749990894221F93E00E
:1005F0009A95F1F748990894221F93E09A95F1F79C
:1006000049990894221F93E09A95F1F74899089424
:10061000221F93E09A95F1F749990894221F4130DF
:1006200071F453E000000000351718F000000000DE
:10063000000048990894221F3A9519F605C0000059
:10064000000000000000F5CF2D93BF91AF913F91C6
:100650002F910F900FBE0F904F915F9118950F92B1
:100660000FB60F922F933F93AF93BF93A4E6B5E0DD
:10067000221B30E19FEF9A9539F34899FCCF489BB4
:10068000FECF99B190FDFDCF91FD08942D932227C7
:10069000221F99B191FDFDCF90FD0894221F00000B
:1006A000000099B190FDFDCF91FD0894221F00003C
:1006B000000099B191FDFDCF90FD0894221F00002C
:1006C000000099B190FDFDCF91FD0894221F00001C
:1006D000000099B191FDFDCF90FD0894221F00000C
:1006E000000099B190FDFDCF91FD0894221F0000FC
:1006F000000099B191FDFDCF90FD0894221F3A951D
:1007000001F6A2CF00000000BCCFAF92BF92CF9203
:10071000DF92FF920F931F93CF93DF936C01EB0156
:100720008A0145D2F82E811124C00115110539F036
:10073000F80180819181C81BD90BC80ED91EB12C3C
:10074000A12C2097B1F08091E80085FD22C0809116
:10075000E8008E778093E80005D501151105A1F01A
:10076000F80180819181A80EB91EB182A08285E036
:10077000F82E8F2DDF91CF911F910F91FF90DF9079
:10078000CF90BF90AF90089512D28823D1F2F82E67
:10079000F0CFF60181916F018093F1002197FFEF77
:1007A000AF1ABF0ACECFAF92BF92CF92DF92FF9225
:1007B0000F931F93CF93DF936C01EB018A01F7D165
:1007C000F82E811124C00115110539F0F80180813E
:1007D0009181C81BD90BC80ED91EB12CA12C209712
:1007E000B1F08091E80085FD22C08091E8008B7710
:1007F0008093E800B7D401151105A1F0F8018081BC
:100800009181A80EB91EB182A08285E0F82E8F2DAD
:10081000DF91CF911F910F91FF90DF90CF90BF900C
:10082000AF900895C4D18823D1F2F82EF0CF8091F3
:10083000F100F60181936F012197FFEFAF1ABF0A14
:10084000CECFFC0180911305909114058617970770
:10085000A0F06115710529F49091E8009E779093BE
:10086000E80090E06115710551F4911108C0809184
:10087000E80082FF34C080E00895BC01F2CF80918F
:100880000C058823C1F18530C1F18091E80083FD1A
:1008900030C08091E80082FDEACF8091E80080FFBF
:1008A000E1CF8091F3002091F200382F611571059E
:1008B00019F02034310558F091E02034310509F069
:1008C00090E02091E8002E772093E800CBCF819133
:1008D0008093F100615071092F5F3F4FE7CF809106
:1008E0000C05882341F0853041F08091E80083FFBA
:1008F000BECF81E0089582E0089583E00895FC0171
:100900006115710529F49091E8009B779093E800B8
:100910006115710531F48091E80080FF1EC080E010
:10092000089580910C05882311F18530E1F08091C4
:10093000E80083FD1AC08091E80082FFE9CF809132
:10094000F3002091F200382F232BE9F28091F1007F
:1009500081936150710999F7D6CF80910C05882356
:1009600031F08530C1F683E0089581E0089582E09A
:100970000895FC018091130590911405861797073F
:10098000A0F06115710529F48091E8008E778093BD
:10099000E80090E06115710551F4911108C0809153
:1009A000E80082FF35C080E00895BC01F2CF80915D
:1009B0000C058823C9F18530C9F18091E80083FDD9
:1009C00031C08091E80082FDEACF8091E80080FF8D
:1009D000E1CF8091F3002091F200382F611571056D
:1009E00019F02034310558F091E02034310509F038
:1009F00090E08091E8008E778093E800CBCF8491DF
:100A00008093F1003196615071092F5F3F4FE6CF1F
:100A100080910C05882341F0853041F08091E800F9
:100A200083FFBDCF81E0089582E0089583E00895BB
:100A3000EF92FF920F931F93CF93DF937C01EB0113
:100A4000809113059091140586179707C0F02097A1
:100A500029F48091E8008E778093E80080E0209769
:100A600081F481110EC08091E80082FF3DC080E0DA
:100A7000DF91CF911F910F91FF90EF900895EC01BE
:100A8000EDCF90910C059923D9F19530D9F1909142
:100A9000E80093FD33C09091E80092FDE4CF90917F
:100AA000E80090FFDCCF8091F3000091F200182F56
:100AB000209719F00034110558F081E00034110539
:100AC00009F080E09091E8009E779093E800C7CF0E
:100AD000C7010E941A3A8093F1008FEFE81AF80AD2
:100AE00021970F5F1F4FE4CF80910C05882341F0C1
:100AF000853041F08091E80083FFB5CF81E0B8CF29
:100B000082E0B6CF83E0B4CF982F973028F08F7073
:100B10008093E90081E008959093E900242F762FD7
:100B200050E0981731F07091EC002091ED00509159
:100B3000F00021FD02C09F5FE8CF3091EB003E7FC7
:100B40003093EB003091ED003D7F3093ED0030911C
:100B5000EB0031603093EB007093EC002093ED00DC
:100B60005093F0002091EE0027FDE5CF80E008953E
:100B700080910D0587FF13C08091E80082FF06C0B9
:100B80008091E8008B778093E80004C080910C0589
:100B90008111F2CF089580910C058823D9F38091BB
:100BA000E80080FFF8CF8091E8008E77ECCF2091AD
:100BB000E4003091E50095E6A9012091EC00822F38
:100BC000817020FF06C08091E80080FF06C080E0B1
:100BD00008952091E80022FD1AC080910C05882319
:100BE00089F0853089F08091EB0085FD0FC0209160
:100BF000E4003091E50042175307F9F29150E1F615
:100C000084E0089582E0089583E0089581E00895E6
:100C100067D06ED0E0EEF0E0808181608083E8ED07
:100C2000F0E080818F77808319BCA7EDB0E08C91D4
:100C30008E7F8C9380818F7E808310920B05089528
:100C40000F931F93CF93DF934BD052D0C8EDD0E0DA
:100C500088818F77888388818068888388818F7D69
:100C6000888319BC10920C051092080510920A0591
:100C70001092090500EE10E0F80180818B7F8083DF
:100C800088818160888342E360E080E03DDFE1EEBF
:100C9000F0E080818E7F8083E2EEF0E080818160F1
:100CA0008083808188608083F80180818E7F80834B
:100CB000888180618883DF91CF911F910F91089582
:100CC000E8EDF0E080818F7E8083E7EDF0E08081C9
:100CD0008160808384E082BF81E080930B05B0CF88
:100CE000E8EDF0E080818E7F80831092E20008952D
:100CF0001092DA001092E10008951F920F920FB641
:100D00000F9211242F933F934F935F936F937F9391
:100D10008F939F93AF93BF93EF93FF938091E100E5
:100D200082FF0BC08091E20082FF07C08091E1004A
:100D30008B7F8093E1000E94512A8091DA0080FF2E
:100D400019C08091D80080FF15C08091DA008E7F95
:100D50008093DA008091D90080FF8DC080E189BD49
:100D600082E189BD09B400FEFDCF81E080930C05CE
:100D70000E94552A8091E10080FF18C08091E20016
:100D800080FF14C08091E2008E7F8093E20080910A
:100D9000E20080618093E2008091D80080628093BD
:100DA000D80019BC85E080930C05DBD18091E1006F
:100DB00084FF2AC08091E20084FF26C080E189BDC3
:100DC00082E189BD89B5982F917080FFFBCF80911A
:100DD000D8008F7D8093D8008091E1008F7E809332
:100DE000E1008091E2008F7E8093E2008091E2003A
:100DF00081608093E20080910805882309F441C056
:100E000084E080930C05ADD18091E10083FF22C086
:100E10008091E20083FF1EC08091E100877F809374
:100E2000E10082E080930C05109208058091E100BA
:100E30008E7F8093E1008091E2008E7F8093E200BC
:100E40008091E20080618093E20042E360E080E014
:100E50005BDE87D1FF91EF91BF91AF919F918F9111
:100E60007F916F915F914F913F912F910F900FBEA6
:100E70000F901F90189519BC10920C050E945B2AC8
:100E800079CF8091E30087FD93E090930C05BBCF71
:100E90001F93CF93DF93CDB7DEB7AB970FB6F89420
:100EA000DEBF0FBECDBF8DE095E02091F100FC01CB
:100EB0002193CF01F5E085319F07B9F70E94662A9B
:100EC0008091E80083FF11C090910D0580910E057F
:100ED000853009F4BEC008F5813009F487C0882345
:100EE00009F45CC0833009F481C08091E80083FF7D
:100EF0000AC08091E800877F8093E8008091EB0032
:100F000080628093EB00AB960FB6F894DEBF0FBE05
:100F1000CDBFDF91CF911F910895883009F4E1C0D2
:100F2000893009F4EBC0863001F790589230E8F62A
:100F300080910F05909110058C3D23E0920709F0F8
:100F4000AAC083E08A838AE289834FB7F894DE01DE
:100F5000139620E03EE051E2E32FF0E0509357007B
:100F6000E49120FF03C0E295EF703F5FEF708E2F9A
:100F700090E0EA3008F48DC0C7968D939D932F5F63
:100F8000243151F74FBF8091E800877F8093E800BC
:100F90006AE270E0CE01019654DC98C0903899F076
:100FA000923809F0A2CF809111058F70873008F038
:100FB0009CCF8093E9008091EB0085FB882780F926
:100FC0001092E90006C08091090590910A059111DF
:100FD00082609091E800977F9093E8008093F10001
:100FE0001092F1008091E8008E77B7C0992309F440
:100FF000A4C0923009F079CF90910F059111A8C04B
:10100000909111059F702FEF290F263008F06DCFBA
:101010009093E9002091EB0020FF9AC0833031F4D7
:101020008091EB0080628093EB0092C08091EB0096
:1010300080618093EB0021E030E001C0220F9A959F
:10104000EAF72093EA001092EA008091EB008860B2
:10105000EACF91114ACF10910F051F778091E300DD
:101060008078812B8093E3008091E800877F8093D4
:10107000E8007EDD8091E80080FFFCCF8091E300F6
:1010800080688093E30082E0111183E080930C0577
:101090002CCFC09672CF60911105709112059E0100
:1010A000255D3F4FAE014F5F5F4F0E94732FBC0124
:1010B000892B09F41ACF8091E800877F8093E8009C
:1010C0002BA589819A81211107C053DC8091E8000A
:1010D0008B778093E80009CF213009F05DCFA8DC41
:1010E000F5CF903809F001CF8091E800877F809399
:1010F000E800809108058093F10074CF9111F5CE3E
:1011000090910F05923008F0F0CE8091E800877F33
:101110008093E800909308052BDD809108058823D3
:1011200011F084E005C08091E30087FDFACF81E0F3
:1011300080930C050E945C2AD8CE90910F059130C7
:1011400009F0D3CE91E0833009F090E090930A0546
:101150001092E9008091E800877F8093E80008DD25
:10116000C4CE0895CF9380910C05882399F0C09147
:10117000E900CF709091EC00892F817090FD80E89C
:10118000C82B1092E9008091E80083FD81DECF70CA
:10119000C093E900CF910895CB017093130360933E
:1011A000120365E00C94162A9B018093140364E0FB
:1011B000C9010C94162A289887EC90E00197F1F762
:1011C00000C000000895289A8FE891E00197F1F798
:1011D00000C0000008958EBD0DB407FEFDCF8EB592
:1011E00095E89A95F1F700000895EF92FF920F931A
:1011F0001F93CF93DF937C01162F042FDCDFD0E009
:10120000C0E0F701EC0FFD1F84911F3F19F01C1384
:1012100001C0802FE0DF2196C930D10591F7DF9121
:10122000CF911F910F91FF90EF90CDCF482F63E0AA
:101230008CEA90E0DACFCF93DF9310925D05C0E0A7
:101240008CB580648CBDB7DF81E0C5DF82E4C3DF8D
:10125000D82F80E0C0DF80E0BEDF80E0BCDF8CB54F
:101260008F7B8CBDB0DF8EEF8D0F8D3FC0F4D234FD
:10127000B1F081E08093FC0280935D058FE79EE3EF
:101280000197F1F700C0000080915D05811103C056
:1012900088988098D0E08D2FDF91CF9108958FE5C9
:1012A0009AEE0197F1F700C00000C43040F08CB511
:1012B00083608CBDCF5FC63009F0C2CFE5CFC230AE
:1012C000C8F38DB58E7F8DBDF5CFEF92FF921F9342
:1012D000CF93DF93CDB7DEB7A0970FB6F894DEBFFC
:1012E0000FBECDBF8CB580648CBD65DF10E08091F2
:1012F000B9061817E8F08CB58F7B8CBD64DF1091B0
:10130000B906412F50E0BE016F5F7F4F87E995E03E
:101310000E940A3A10939605A0960FB6F894DEBF85
:101320000FBECDBFDF91CF911F91FF90EF90089539
:10133000E12EF12CF701EA56FA4F80814CDFE1E013
:10134000F0E0EC0FFD1FEE0DFF1D80831F5FCFCF80
:10135000E091BB06F091BC060190F081E02D09956B
:10136000889A809A84B1876084B923982B988DE7F6
:101370008CBD8DB581608DBD80916305811103C0E9
:101380008DE08093630580917905811103C08EE023
:101390008093790580919C06811103C083E180933D
:1013A0009C0680917605811103C084E180937605C7
:1013B00010925805109259051092FB0286EF809307
:1013C000FA0280915B05811103C084E60C94C52E5E
:1013D00008950F931F93CF93DF9381E0809360056F
:1013E0008CB580648CBDE7DE81E0F5DE82E4F3DE5F
:1013F0008093FE0280E0EFDEC82F81E0209112038F
:1014000030911303232B09F480E08195E4DE80936F
:10141000000380911403DFDE809301038091FE02BC
:10142000893759F0982F9F7D933539F0873729F008
:10143000833E71F48FE78093FE02CC23A1F0CA357E
:1014400091F0CF3F09F079C181E080935B05E8C05E
:10145000833211F483E3EFCF8DB58E7F8DBD83E7AB
:1014600080936105EACF8091FE0290916105891712
:1014700041F091E0813409F48AC09093FC0210920B
:101480005F0580936105813409F084C081E0809319
:1014900003038093020397DE8091FC02882359F1B5
:1014A0001092FC028BEF93E00197F1F700C000006F
:1014B00080916105813409F48BC081E0B7DE40E0A2
:1014C0006FEF80ED90E091DE40E06FEF80ED90E017
:1014D0008CDE40E06FEF89ED90E087DE40E06FEF5B
:1014E0008EEB90E082DE80E0A1DE8FE99FE0019745
:1014F000F1F700C000008CB58F7B8CBD909101038B
:101500009095292F229560E062276D73622720FB5A
:1015100063F922FB60F923FB62F9262F8091000317
:10152000809530E080FB34F983FB35F9232B209341
:101530004B05937030E081FB36F982FB37F9932B32
:1015400090934C0570E084FB72F985FB75F986FB7E
:1015500073F987FB74F9872F709356059091FA02FF
:1015600019160CF469C09F5F9093FA0274FF67C06C
:101570002F3F09F464C010925F0592E09093FA0245
:101580008F7E809356058BE48093610558C09093BD
:101590005F0577CF893759F4C2E0D3E002E113E069
:1015A00080E019DE89930C171D07D1F774CF80E016
:1015B00012DE8093020380E00EDE8093030380E05E
:1015C0000ADE8093040380E006DE8093050363CF88
:1015D00081E02CDE40E06FEF8EEB90E006DE41E034
:1015E00063E087EC90E001DE80E020DE81E0F3DD67
:1015F00082E4F1DD182FC7E0D0E080E0ECDD219738
:10160000E1F7113409F059CF76CF1092FB020DB4F7
:1016100000FE0EC08DB58E7F8DBD81E080935C0590
:101620008CB58F7B8CBDDF91CF911F910F91CBCD6E
:101630008CB583608CBDF1CF923009F4A1CF20919D
:10164000020390910303622F690F7727771F62309F
:10165000710579F48CB58F7B8CBDB5DD8FE193E09E
:101660000197F1F700C00000DF91CF911F910F911A
:101670000895809161058F3741F0309104033093D4
:101680004E053091050330934F05209351059093FB
:1016900052051092530510925005893791F5A6E036
:1016A000B3E0EDE9F6E08D91819396E0E93AF90730
:1016B000D1F7E0916305E53131F0F0E0E350FD4F03
:1016C000808180935405E0917905E53131F0F0E0B7
:1016D000E350FD4F808180935505E0919C06E531F4
:1016E00031F0F0E0E350FD4F808180935005E091B0
:1016F0007605E53131F0F0E0E350FD4F80818093D5
:1017000053058CB58F7B8CBD5EDD8CB583708330CB
:1017100069F08DB59091FA02923031F090916105A7
:1017200080958170933719F486E001C08EE0DF91D7
:10173000CF911F910F910C94532F8091FB028F5FDB
:10174000843609F462CF8093FB0267CF80E091E09A
:10175000089528E030E040E891E07CEF63E0582F06
:10176000542389F05BB1592B5BB95BB153605BB912
:10177000EBB1592F50955E235BB9962746952150C2
:10178000310969F70895592F57275BB95BB15C7F21
:10179000F3CFEF92FF921F93CF93DF93EC017C0185
:1017A000E60EF11C10E0CE15DF0539F4812FDF9134
:1017B000CF911F91FF90EF9008958991CADFFE01AC
:1017C000319780811827EFCF8BB183608BB98AB1B5
:1017D00083608AB98BB183608BB9589888E022E026
:1017E0009BB192279BB98150D9F78BB183608BB99C
:1017F00008958BB183608BB98AB183608AB98BB14C
:1018000083608BB9599884E021E09BB192279BB902
:101810008150D9F78BB183608BB90895D5DF68E02B
:1018200088E391E0B6DF95DFE4CFCEDF64E084E3C8
:1018300091E0AFDF8EDFDDCF80911D03882349F07B
:1018400010925F0580911B03811102C080E1089511
:101850008EE30895CB012FEF20931A037093210399
:1018600060932003009719F065E00C94162A089500
:101870009B0180931A0370931F0360931E03672BD1
:1018800021F064E0C9010C94162A08959DDF60914F
:10189000B90686E995E07DDF5CDFABDFE6E9F5E0E0
:1018A00088E080838FEF818381E00C94532FCF9366
:1018B000C82F833019F481E0FADFC2E085DFC093DE
:1018C000260164E084E291E064DF43DF92DF8BB1C4
:1018D00083608BB98AB18C7F8AB982E00E94532FD2
:1018E00065E084E690E00E94162A8BB183608BB994
:1018F0008AB183608AB9CF910895CF93C82F64DFEE
:10190000C09323016CE088E191E043DF22DF71DFC7
:101910008BB183608BB98AB18C7F8AB987E795E0F8
:101920000197F1F700C00000CF9108951F93CF9366
:10193000DF93182FD42F62956695677009F461E0E4
:10194000C62FC295C07F40DF10932A0187E2103175
:1019500009F48FE080933101C0933201D295D07F9A
:10196000D09333016CE088E291E013DFF2DE41DFD7
:101970008FEA94E00197F1F700C00000DF91CF916A
:101980001F910895CF937894E091BB06F091BC0627
:101990000190F081E02D09958BB183608BB98AB1FC
:1019A00083608AB910921D0310921C0310921503D4
:1019B000109222031092230310921B0310926505CC
:1019C00010926705C1E0C09319031092180310929A
:1019D0001603109221031092200310921F031092FD
:1019E0001E0323DF8BB183608BB98AB18C7F8AB9E8
:1019F00082E00E94532F8BB183608BB98AB18360E0
:101A00008AB90CDF8BB183608BB98AB18C7F8AB9BC
:101A10001092690082E08DBBEBE3F1E03197F1F7C2
:101A200000C000001DBA1DBA90916705953521F1DF
:101A3000911117C0E3E0F1E03197F1F700C0000029
:101A40008DBB8BE391E00197F1F700C000001DBA58
:101A50001DBAC0931B0380911D0390916505892BCE
:101A600059F081E080931D0380937B05EFE1F3E063
:101A70003197F1F700C00000CF9108950F931F93A5
:101A8000CF93DF9381E08093600510926F051092F1
:101A900067058BB183608BB98AB183608AB9BEDE7A
:101AA0008BB183608BB98AB18C7F8AB980911B031B
:101AB000882389F18FE891E00197F1F700C00000D9
:101AC00080916605837080936405ECE6F5E084E61A
:101AD00095E02085208331978E179F07D1F780915D
:101AE0006705811131C080911C0381111FC0C1E0C5
:101AF000C0931C039ADE8BB183608BB98AB18C7F53
:101B00008AB982E00E94532FC0935C05DF91CF9188
:101B10001F910F91089582E08DBB8BE391E00197B7
:101B2000F1F700C000001DBA1DBAD9CF81E0809343
:101B30005B0510921803109216038BB183608BB96A
:101B40008AB183608AB9E2CF10921C039BB1936083
:101B50009BB99AB19C7F9AB930916405932F937089
:101B60009093170350916505593C18F08E7F809330
:101B7000670540916605493C28F0809168058E7F95
:101B80008093680590916805892F809520E080FBFF
:101B900027F981FB21F982FB20F983FB25F980914C
:101BA0006705809560E080FB66F981FB63F982FB45
:101BB00062F983FB64F9862F822B80934B0533FFF8
:101BC000A2C089E4809361059095959595959C7345
:101BD00090935605509350054093530580916905A5
:101BE00090916A05982789279827909352058093AA
:101BF000510580916B0590916C059827892798274E
:101C000090934F0580934E0587E592E00197F1F799
:101C100000C0000080911E0390911F0320912003BB
:101C200030912103822B932B892B09F49FC0809143
:101C30001803882351F060911A038091190393E0EF
:101C400089278093190341E071DE80911603882370
:101C500049F02091200330912103232B19F042E019
:101C60006FEF64DE80911603882351F020911E03EC
:101C700030911F03232B21F041E060911A0356DEBF
:101C800080917B05813069F58091180380FF29C020
:101C900082E00E94532F10927B0596DD6CE08CE071
:101CA00091E077DDD82FC0E003E08C2F802790E013
:101CB00080569F4F0E941A3A182F4BDDD127CF5FD5
:101CC000C03C99F78D2F45DD94DD8BB183608BB9D6
:101CD0008AB18C7F8AB98FEA94E00197F1F700C04E
:101CE000000087E592E00197F1F700C000008091C5
:101CF00061058A3409F00ACF8FE0DF91CF911F91FF
:101D00000F910C94532F84FF03C021E020932303F1
:101D10002091230397FD09C031E030932203222351
:101D200081F023E2209361050CC030912203311130
:101D3000F6CF222331F02AE42093610521E020939D
:101D4000150320916105233261F4292F2095322F4C
:101D50003295337030934C05207C822B80934B0559
:101D600033CF2A3409F030CF8F7AF8CF8091170320
:101D7000882369F090911803891749F0892797DD26
:101D80008091180390911703892B809318039091E9
:101D90001703933051F020911803921731F081E02E
:101DA000911180E082238093180380911603909113
:101DB0006105993471F484FD63CF80E178DD81E0C1
:101DC0009CDD82E09ADD809116038061809316038A
:101DD00057CF8F7EFBCF80E491E00895CF93C82F3B
:101DE000CB0164E00E94162ACC2351F081E080935D
:101DF000260386E080932503C0932403CF910895A2
:101E00001092260384E08093250310922403F6CFDA
:101E1000E5CF0C948B281F93CF93DF93CDB7DEB71C
:101E200028970FB6F894DEBF0FBECDBF81E0809338
:101E30006005198261E0CE0101960E94C5278330BA
:101E400071F08FE891E00197F1F700C0000061E0C8
:101E5000CE0101960E94C52711E0833009F410E0FD
:101E6000809161058231F1F480E3898380912503BB
:101E70008A83809124038B8363E0CE0101960E94C4
:101E8000C5278830E9F081E01123B9F080935B0524
:101E900028960FB6F894DEBF0FBECDBFDF91CF916D
:101EA0001F91089580E4898383E08A8381E0909183
:101EB00026039111E0CF80E0DECF80935C05E8CF70
:101EC0008091180580934E059091190590959093F7
:101ED0004F0580911A058093510580911B058095CF
:101EE0008093520580911C058093500580911D05BB
:101EF0008093530580911605880F20E02827257DC3
:101F0000282782FB20F984FB22F9822F20911705D4
:101F100030E032273F7A322725FB37F9830F809351
:101F20004B0580E020FB84F921FB85F922FB83F936
:101F300023FB82F98093560580916105823131F44B
:101F4000909590934E0580E880934F0580914E05C3
:101F500090915105892B09F09BCF8091520590916A
:101F60004F0589238F3F09F093CF80E880934F0579
:101F700080934E05809350058093520580935105C0
:101F800087CFE091BB06F091BC060190F081E02D77
:101F900009950E94C2271092260384E080932503AE
:101FA0001092240308958CE491E0089508959B0114
:101FB00070934B0360934A0390916401953089F0CC
:101FC000992379F0882339F082E0933039F464E082
:101FD000C9010C94162A9130D1F384E080936401F6
:101FE000F6CF0895E4CF0C948B2893E090932703C9
:101FF0008093280360932903642F70E040E250E04F
:102000008AE293E00E94133A63E287E293E00E943F
:10201000C52791E0813009F490E0892F81950895DA
:10202000482F6BE180ECE1CF8091160520E084FB26
:1020300025F985FB24F986FB20F987FB21F990918E
:102040001705392F330F40E04327437B432735FBE8
:1020500047F9242B20934B0520E090FB21F993FBBB
:1020600020F920934C0540E080FB45F981FB44F9C1
:1020700082FB43F983FB42F9409356058091180592
:102080008F3F11F4109218058091180581588093A4
:102090004E05809119059FE7892780934F05089584
:1020A000CF93C1E0C093600580911505882329F086
:1020B0008DE280936105CF910895C093270361E07D
:1020C00087E293E00E94C527811103C0C0935B059E
:1020D000F2CF843011F0C0935C05A6DF87EC90E06E
:1020E0000197F1F700C000001092270361E087E23A
:1020F00093E00E94C527833011F010926401809113
:102100001805813099F4809164018530A9F410920A
:10211000640140E861E080E868DF882371F140E80D
:1021200061E080E862DF811103C0C5CF823021F415
:1021300085E080936401BFCF80916401833070F4A7
:10214000882339F380914A0390914B03892B09F43A
:10215000B2CF81E065DF8111AECF17C0853008F0C6
:10216000AACF80914A0390914B03892B09F0A3CF0A
:1021700080E056DF81119FCF0CC080914A0390917F
:102180004B03892B21F081E04BDF83E0D2CF80E04D
:1021900047DF81E0CECF88E591E008950895089566
:1021A000E091BB06F091BC060190F081E02D09950D
:1021B0008BB183608BB9089588EB9BE02091BC00C4
:1021C00027FD02C00197D1F78091B900887F08955B
:1021D000883321F484E88093BC00089584E9FBCF20
:1021E0001F93CF93DF93182FD62FC4EAC093BC0060
:1021F000E3DF883051F5C093BB00C4E8C093BC0056
:10220000DBDF8831E1F41093BB00C093BC00D4DF66
:102210008832C1F4D093BB00C093BC00CDDF8832BC
:1022200089F484E98093BC0080E0EFE1F3E031972A
:10223000F1F700C00000DF91CF911F910895C8DF32
:1022400082E0F3CFC5DF83E0F0CF81E0EECFEF9205
:10225000FF920F931F93CF93DF93E82E8B01C42F30
:10226000D4EAD093BC00A8DF883009F05BC0D093DB
:10227000BB0094E8F92EF092BC009EDF8831A9F5EE
:10228000E092BB00F092BC0097DF8832B9F584E998
:102290008093BC008FE193E00197F1F700C000004C
:1022A000D093BC0089DF803161F585EA8093BB0063
:1022B00084E88093BC0080DF803441F5D4E884EC6E
:1022C000F82EC15038F029F1F092BC0075DF877FFD
:1022D000803511F184E98093BC00EFE1F3E03197A0
:1022E000F1F700C0000080E002C072DF82E0DF9101
:1022F000CF911F910F91FF90EF90089569DF83E0D8
:10230000F6CF883091F264DF84E0F1CF61DF85E0C1
:10231000EECFD093BC00DACF8091BB00F80181935F
:102320008F01CFCF81E0E3CFCF93DF93CDB7DEB77F
:1023300060970FB6F894DEBF0FBECDBF84E38093E5
:10234000B8008091B9008C7F8093B90080917101B1
:10235000811139C065E580EF43DF882359F0109281
:10236000BC0060960FB6F894DEBF0FBECDBFDF9104
:10237000CF91089560E08BEF33DF8111F0CF42E021
:10238000BE016F5F7F4F8EEF62DF8111E8CF8A81E0
:1023900080937201811107C08DE08093610581E017
:1023A00080937101DCCF813011F48FE1F6CF83305F
:1023B00011F483E4F2CF853011F480E2EECF823164
:1023C00071F785E4EACF813051F68091610546E0EE
:1023D0008F3109F448E0BE016F5F7F4F80E037DF47
:1023E000882349F081E080935B0580EF8093720140
:1023F00010927101B4CF20917201233041F008F0A6
:102400009EC0222309F4A1C0213009F0A8CF9981F0
:102410002A818B814C8130917301332309F4F3C0FD
:102420003D8190934E05809580934F0520935105F3
:10243000409540935205309350058E81809353050B
:10244000E7E0A6E081E090E08C0F9D1F8A0F911DD0
:10245000DC012C91922F909530E091FB37F992FBA3
:1024600035F994FB34F995FB36F9932FF0E0A1E0B0
:10247000B0E0AC0FBD1FAE0FBF1F8C91809530E058
:1024800083FB33F984FB31F985FB32F986FB30F9A4
:10249000932B90934B0540E082FB41F987FB40F979
:1024A000842F40934C0523FD05C090914D05946009
:1024B00090934D0510925605A1E0B0E0AC0FBD1F02
:1024C000AE0FBF1F9C9190FD03C034E030935605C2
:1024D00027FD05C03091560530623093560591FDB9
:1024E00005C03091560530613093560526FD05C074
:1024F00020915605286020935605209161052334CC
:1025000009F0C6C020915005222309F4D8C084E404
:102510008093610510925F0580914E0581111FCF58
:1025200080914F058F3F09F01ACF80E880935205C4
:102530008093510580934F0580934E0510CF213134
:1025400009F465CF223109F00ACF898180934E05C5
:102550008A81809580934F054E81842F809583706A
:1025600090914B05892B80934B056C81842F90E0D3
:10257000FC0175E0EE0FFF1F7A95E1F7E078362F4A
:102580003695E32BE0935205223109F4E8CE2D81F4
:1025900054E0259F9001112442954695469543703D
:1025A000242B2A5F3109AC015595479555954795E0
:1025B00043705527EB8174E0E79FF00111244E2B07
:1025C0005F2B4A5F51095695479540935105B4E0FA
:1025D00095958795BA95E1F78370992744E0649FB4
:1025E000B0011124862B972B8A5F910996958795C8
:1025F00080935205369527952093550510925305E3
:1026000010925005ACCE392F330F330F30934E0557
:1026100030E0B901660F771F660F771F60956093F2
:102620004F0565E0359527956A95E1F726709695F3
:10263000969596959871292B982F991F9927991FF0
:10264000292B220F220F220F20935105982F990F2B
:10265000990F990F90959093520558E0459F9001DE
:1026600011242093530590E095958795959587952E
:1026700088719927429546954770842BE3E0880F2F
:10268000991FEA95E1F780935005E5E0A4E0DACEE2
:10269000243409F04AC08091510580588093510537
:1026A0008091530580588093530580914B0581FBA1
:1026B000992790F9892B8D7F80934B052DCF209101
:1026C0004E0510925F052093510520914F052093F0
:1026D00052052091530520934F0520E82093500583
:1026E0002093530520934E0520914B05207F8E7F2C
:1026F00080934C05909550E093FB53F995FB50F96E
:1027000096FB51F997FB52F9952F922B90934B051D
:1027100021E030E02C0F3D1FE20FF31F908194FD6C
:10272000FBCE826080934C05F7CE2F3109F0F4CEBA
:1027300090914B059F3F09F0EFCE833009F0ECCE2E
:1027400010927301E9CEF0DD80917201803F59F063
:10275000813031F463E08EEF43DD809161050895AF
:1027600010927301FACF80E0089585E691E0089514
:102770000895E091BB06F091BC060190F081E02D38
:10278000099510924D0310924C0384E08093D90177
:10279000E0E8F1E090E1918B87838BE290E0928317
:1027A000818310925803089580935703089580936E
:1027B00056030895E0914C03F0914D03A381B48139
:1027C0008C919781892B8C93A285B3858C9196856A
:1027D000892B8C938081813051F4A085B1859C91A7
:1027E0008685809589238C9382E00C94532F8230C8
:1027F000C9F4519A599A579A5F9A569A5E98509A84
:102800005898E0914C03F0914D03A181B2819C91C5
:102810008781809589238C93A085B1858C9196853D
:10282000892BE1CF833081F4539A5B98A0914C03BC
:10283000B0914D031896ED91FC91199780811E96E9
:102840009C91892B8083D0CF843071F6569A5E9804
:10285000509A589A259AA0914C03B0914D0318961E
:10286000ED91FC91199790811E968C91809589230A
:10287000E9CF90E0981301C0089525E02A95F1F77B
:1028800000009F5FF7CFDF92EF92FF920F931F93AD
:10289000CF93DF93082FF62EE22EA0914C03B09138
:1028A0004D031896ED91FC9119971E968C9190818D
:1028B00041114EC0892B808385E38A95F1F7000092
:1028C000CEE4D3E010E0025B1C4F88E0D82E988164
:1028D000990F9883E0914C03F0914D0381E0E81249
:1028E00008C0A785B0898C912189822311F091605D
:1028F0009883A181B2819C918781809589238C9353
:102900008F2DB7DFE0914C03F0914D03E11009C02A
:10291000A785B0898C919189892319F0888181607C
:102920008883A181B2818C919781892B8C938F2D83
:10293000A0DFDA94D110CBCF21960C171D0729F612
:10294000DF91CF911F910F91FF90EF90DF9008954D
:10295000413089F4809589238083862F8ADFA09176
:102960004C03B0914D031896ED91FC91199780811D
:102970001E969C919FCF892B8083862F7ADFA09112
:102980004C03B0914D031896ED91FC9119979081ED
:102990001E968C91809589238ECFCF93DF9384EA06
:1029A00091E090934D0380934C0304DF8FE99FE007
:1029B0000197F1F700C00000C3E0A0914C03B09173
:1029C0004D031196ED91FC911297808117969C9181
:1029D000892B80838FEC97E00197F1F700C000000E
:1029E000A0914C03B0914D031196ED91FC9112977B
:1029F000908117968C9180958923808320E040E018
:102A000060E082E040DFC150C1F680914E038F7BD1
:102A1000803809F4E0C0ADDE82E991E090934D0387
:102A200080934C03C7DE20E041E062E084E02BDFCE
:102A300080915103803F09F4D0C09BDE88EC91E087
:102A400090934D0380934C03B5DE21E042E067E0B4
:102A500084E019DF80914E038F3349F48091500355
:102A60008F3F69F481E080935803C1E163C08F3FD9
:102A700031F48091500390914F03892BB1F38091F1
:102A80004F038F3F31F480915003811111C0CBE18E
:102A900051C08B3F31F4809150038F3F49F4CFE216
:102AA00049C08C3F29F480915003882309F497C0D2
:102AB00080E28093D9018FE79EE30197F1F700C090
:102AC000000021E042E067E081E0DDDE80914E031E
:102AD000803F09F486C08F3729F082508D3F18F46B
:102AE000CEE128C0C1E0D0E1D093D901E0914C0300
:102AF000F0914D030784F089E02D80818D3E09F42B
:102B000072C037DE86EB91E090934D0380934C03C7
:102B100051DE5E98569A5D9A559A21E042E067E050
:102B200084E0B1DE80914E038F3B41F481E08093DD
:102B30005803CDE48C2FDF91CF9108951ADE80E801
:102B400091E090934D0380934C0334DECC2349F005
:102B500086E485B99FEB9BB984B981E48AB9CFE358
:102B6000E9CFD093910184E0809387018BE290E0DC
:102B7000909382018093810121E042E067E084E04C
:102B800082DE80914E038F3F51F480914F039091EC
:102B90005003892B51F180915103882341F186E044
:102BA0000E94532F82E08093910180E280938701FD
:102BB00085E290E0909382018093810121E042E0E0
:102BC00067E081E060DE80914E0382508D3F08F027
:102BD000B1CFC5E3AFCFC9E1ADCFCAE1ABCFCDE156
:102BE000A9CFC4E2A7CFCCE1A5CFC4E3A3CFC7E46C
:102BF000A1CF1F93CF93DF9380916105893109F0B5
:102C000083C0A0914C03B0914D031196ED91FC91BE
:102C10001297908117968C9180958923808320E06C
:102C200041E060E088E02FDE809161058931C1F5E7
:102C300020914F0380E082278F7C822726FB87F933
:102C400027FB81F930914E03C32FC170C82B259506
:102C50002595237080E031FB84F932FB85F933FB45
:102C600082F934FB83F9382F90E840E850E8A091CE
:102C70004C03B0914D031196ED91FC911297808118
:102C800017966C91862B808380914F038F3F09F0BC
:102C9000D8C281E080935B05DF91CF911F910895A9
:102CA000853259F55091510340915203809153035D
:102CB0008295807F9EEF981B80915503C0E080FB3A
:102CC000C7F981FBC6F982FBC4F983FBC5F93091D2
:102CD0005403E0E0E327EF7CE32736FBE3F937FB1F
:102CE000E2F93E2FF0E0F827F57FF82780FBF2F9B4
:102CF00082FBF0F9CF2B20E0BACF90E840E850E813
:102D000030E020E0C0E0B3CF8A3109F043C020E0DA
:102D100041E065E084E0B7DDC0914E03C0950C2E24
:102D200000FAC5F901FAC4F902FAC6F904FAC2F9BF
:102D300005FAC0F906FAC1F990914F03392F309581
:102D400020E034FB24F935FB23F936FB25F937FB6A
:102D500022F9322F80E291FD80E093FF8064909110
:102D60005103903F09F095CF90E840E850E8D0E853
:102D700020E0C0934B0520934C0580934D05D093E4
:102D800055053093560550934E0540934F0590934B
:102D9000540582CF8C31E9F48AB180638AB935E079
:102DA0003A95F1F700008AB18A608AB98AB18F7CBE
:102DB0008AB900C04D9905C080914B058160809310
:102DC0004B054C9B69CF80914B05826080934B05EE
:102DD00063CF813149F08B3139F08D3129F08F3259
:102DE00019F08D3409F011C121E042E067E082E082
:102DF0004ADD80916105C0914E03C095813111F08B
:102E00008D3461F580E0C4FB85F9C5FB84F9C6FB10
:102E100080F9C7FB81F9C82F80E020E030914E0394
:102E2000309590E030FB95F931FB94F932FB93F942
:102E300033FB92F9392F409158039091610541116C
:102E4000DEC09F3209F4DEC0909150039F3F09F429
:102E500020CF90E840E850E8D0E88BCF8B3119F0D4
:102E60008F3209F0A8C090E0C4FB95F9C5FB94F936
:102E7000C6FB92F9C7FB90F9C92F90914F0390952B
:102E8000E0E094FBE7F995FBE6F996FBE3F997FBA5
:102E9000E1F9CE2B8F3299F590915003292F20958F
:102EA0002F77809151038095382F3078232B022E75
:102EB00000FA26F901FA25F902FA24F904FA22F9AE
:102EC00005FA21F906FA20F930E080FB37F981FB99
:102ED00036F982FB35F983FB34F984FB33F985FB42
:102EE00031F986FB30F9892F90E08095909545E087
:102EF000959587954A95E1F78470832B8FCF8091C4
:102F0000560382958F708093560320915703229524
:102F10002F7020935703F0E18F9FC0011124092ED9
:102F2000000CAA0BBB0B822BAC01BD0152676F6F6B
:102F30007F6F559A5D9AA0914C03B0914D031896FE
:102F4000ED91FC91199780811E969C91892B80832D
:102F50002AE02A95F1F700C0A0914C03B0914D03EF
:102F60001896ED91FC91199780811E969C919095F1
:102F70009823908320E277FF1CC05D9AE0914C0378
:102F8000F0914D03A181B2818C9197819095982306
:102F90009C93A181B2818C919781892B8C93440F52
:102FA000551F661F771F215031F755985D9A80E0B5
:102FB00035CF5D98E3CF8D31F1F430E0C4FB35F9C6
:102FC000C5FB34F9C6FB32F9C7FB33F9C32F209197
:102FD0004F03209580E022FB81F923FB80F924FB3D
:102FE00087F925FB86F9C82B80E026FB80F927FBB3
:102FF00081F9282FDCCF80E020E0C0E00FCF9F32A6
:1030000009F027CF90914F0321CF843209F041C0BE
:1030100080E28093D90121E042E067E081E033DC87
:1030200080914E038F3F09F434CE8095D0E084FB2D
:10303000D7F986FBD2F987FBD3F9C0E085FBC3F94A
:1030400010924E0380E18093D90121E042E067E0D5
:1030500081E019DC80914E03809520E080FB26F909
:1030600083FB25F985FB24F986FB20F987FB21F9F1
:103070002D2BE0E081FBE2F982FBE1F984FBE0F932
:103080008E2F8C2B90E840E850E830E0D0E8C0E08C
:1030900070CE8E3159F580E18093D901E0914C03D7
:1030A000F0914D03A785B0898C9190E08095909523
:1030B000218930E082239323C1E0892B09F4C0E009
:1030C00080E28093D90121E042E067E081E0DBDB30
:1030D00086E00E94532FD0914E03DF3F09F4D9CDF3
:1030E00090E840E850E830E080E042CE843319F0C8
:1030F000873409F056C021E042E067E084E0C3DB9A
:1031000030914E033095C0E034FBC5F935FBC4F96E
:1031100036FBC0F937FBC1F9F0E030FBF5F931FBC4
:10312000F4F932FBF3F933FBF2F93F2F809161059B
:1031300040914F03873479F54095242F2F77909154
:103140005003892F80958078282B022E00FA26F9CB
:1031500001FA25F902FA24F904FA22F905FA21F90B
:1031600006FA20F9892F806880954078842B082EF4
:1031700000FA87F901FA86F902FA85F903FA84F967
:1031800004FA83F905FA81F906FA80F907FA82F957
:10319000909151035BCE80E020E04F3F09F059CE83
:1031A00078CD8F3309F050C0299887EC90E00197D3
:1031B000F1F700C00000299A23B1287089B190E08E
:1031C00081FB90F983FB91F985FB92F9292BE7E5C7
:1031D000F2E03197F1F700C000002A9887EC90E008
:1031E0000197F1F700C000002A9AC3B190E0C3FB39
:1031F00097F989B1E0E081FBE4F983FBE5F985FB10
:10320000E6F98E2F892BE7E5F2E03197F1F700C060
:1032100000002E98E7ECF0E03197F1F700C00000D5
:103220002E9AC3B1C870C82B89B1F0E081FBF0F9C8
:1032300083FBF1F985FBF2F9CF2B90E840E850E8E9
:1032400030E0D0E880E095CD8533C9F580E180930A
:10325000910184E0809387018BE290E0909382015A
:1032600080938101E0914C03F0914D03A785B089D3
:10327000CC91118982E08093910180E28093870153
:1032800085E290E0909382018093810121E042E009
:1032900067E081E0F8DAD0914E03DF3F09F4F9CC22
:1032A0008C2F90E08095909530E081239323C1E0AE
:1032B000892B09F4C0E086E00E94532F11CF90E8DB
:1032C00040E850E830E0D0E880E020E0E0CE84E75D
:1032D00091E0089508950895E091BB06F091BC0631
:1032E0000190F081E02D09958AB180638AB98BB194
:1032F00080638BB95C988BB190E389278BB95C981C
:103300008FE99FE00197F1F700C000008BB1806367
:103310008BB910925A03089589B180958F7025E278
:103320002A95F1F700005C9895E29A95F1F7000074
:1033300099B190959F7025E02A95F1F700008330B0
:1033400019F4911107C008958F3039F49F3059F066
:1033500083E00895933039F408958E3021F49F303E
:1033600011F088E0089580E008951F93CF93DF93D4
:103370008BB180638BB935E23A95F1F70000C9B1A2
:10338000C095C3FB112710F95C9885E28A95F1F787
:1033900000008C2F8770833009F03FC081E080935C
:1033A0005F05D9B1D095DD0FDD0FDC738BB190E3F4
:1033B00089278BB995E29A95F1F70000C9B1C095BC
:1033C000CF7030E0C0FB31F9C1FB37F9C2FB30F9F7
:1033D000C3FB35F9C32F5C9885E28A95F1F70000AD
:1033E0004B9B126089B180958F7090E080FB96F9BD
:1033F00081FB93F982FB92F9C92B4B9B1260809160
:103400005A03843609F0A1C010925A0381E08093D8
:103410005B05DF91CF911F910895CF70CE3009F0F9
:1034200088C081E080935F058BB18F7C8BB930E4DD
:103430003A95F1F75D9A80E48A95F1F789B1880FA2
:103440008E7180935903853008F471C088E08093B1
:10345000610590E0DFEF20E010E0C0E01FC090FFCA
:1034600022C05D9A30E43A95F1F739B13095832F57
:103470008F70953009F44FC028F59230E9F1D0F4FF
:103480009923B1F130E080FB31F981FB37F982FB00
:1034900030F983FB35F99130C1F19F5F8091590379
:1034A0009817E8F2ACCF8BB18F7C8BB980E48A950A
:1034B000F1F7DBCF933059F1943079F7282F22952B
:1034C000207FEBCF9830D1F348F49630B9F39730A2
:1034D00021F7822B809580934F05DFCF9A3071F3CF
:1034E00008F19B30D1F6822B809580935005D5CF83
:1034F000D82FDD0FDD0FD1CF33FD126030E080FB20
:1035000036F981FB33F982FB32F9C32BC6CF33FF87
:10351000C4CF1160C2CF822B809580934E0510924C
:103520005F05BBCF822B809580935305B6CF83E098
:103530008ECFC11107C080915A038F5F80935A03C9
:10354000DFEF5DCFDFEFC0E05ACF8BB180638BB987
:10355000809159038A3011F40E94532FC0934B0578
:1035600010934C05D093560554CF8AED91E0089501
:1035700008950895E091BB06F091BC060190F0819A
:10358000E02D0994EBE5F3E084E0DF011D928A95DC
:10359000E9F780916105873111F08633D9F45D98A0
:1035A000B5E0BA95F1F7000089B18F7080958093EE
:1035B0005C035C9A25E02A95F1F7000089B18F70D1
:1035C000809580935B035C9885E08A95F1F7000015
:1035D0005D9A0895E7E5F3E090E0883111F5549A9B
:1035E0005C985F9890E080E05C9A5C98A6E0AA9571
:1035F000F1F7873050F023B12095227020935C03BF
:1036000001968930910581F708951999F9CFFC0148
:10361000E352FD4F208130915B03232B20935B030A
:10362000EFCF90FF12C05D9AB5E1BA95F1F70000B7
:10363000199B0DC089B180648095819320E22A9501
:10364000F1F79F5F983069F708955D98EDCF89B1E4
:103650008F7BF2CF8AB1806C8AB95E985F9A199B92
:103660000CC080E0EFE5F9E03197F1F700C0000011
:10367000199B67C08F5F8F3FA9F7E091BB06F09160
:10368000BC060190F081E02D09958BB180638BB968
:103690008AB180638AB989B1803F09F47CC0E09126
:1036A000BB06F091BC060190F081E02D0995559A7A
:1036B0008AB1806C8AB95E985F9A80915B03803290
:1036C00019F086E90E94C52E5DDF80915B038C3284
:1036D00019F08E52823020F480915D0385FD5DC02B
:1036E000FFEF29EF80E0F15020408040E1F700C07B
:1036F00000005D9890E39A95F1F75D9A8BEF199B26
:1037000002C0815041F54C9B2BC0E091BB06F0916B
:10371000BC060190F081E02D0995559A5D9A8AB119
:10372000806C8AB95E985F9A82E00E94532F88E18C
:103730008093610527DF80915C03823021F180E076
:10374000089581508E3F08F098CF8FEF199921C0CE
:103750008150E1F792CFE5E0EA95F1F70000CFCF95
:103760001999D3CFFAE6FA95F1F700C04C9BCDCF6B
:103770001999CBCF20E52A95F1F74C99C6CF199B23
:10378000C4CF8EE4089580915B038111D8CF88E186
:10379000089587E0089587E1089584E10895BF9230
:1037A000CF92DF92EF92FF920F931F93CF93DF930D
:1037B000CDB7DEB72C970FB6F894DEBF0FBECDBFE6
:1037C00080916105873009F050C091E001C09F5F92
:1037D00023B1822F827021FDFACF913029F021E0B0
:1037E0009E3F09F020E0922F21E0199B25C0213057
:1037F00011F02E3F09F49F5F21E033B1432F427057
:10380000C42E31FD1CC0213011F02E3FD1F4923076
:10381000C1F481E080935B052C960FB6F894DEBF6F
:103820000FBECDBFDF91CF911F910F91FF90EF9011
:10383000DF90CF90BF9008952F5F89B1D6CF2F5FD3
:10384000DCCF99B184FB112710F921E01227829572
:10385000807F9F70892B80935505B12CD12C80E8F7
:10386000E82E00E890E8F92EAFC0873111F08633DA
:10387000B9F588DE87E18093610580915B038F70E5
:1038800010E08F3079F486E38093610510915C033A
:1038900080E08127837F812710FB87F911FB86F960
:1038A000182F70DE90915C0320E090FB21F991FBD2
:1038B00020F992FB24F993FB25F980915B0340E00A
:1038C00080FB42F981FB45F982FB43F983FB44F914
:1038D000B42E89B18F70C82E09F09BCF122BBECFAA
:1038E0008831C9F45F9A89B18095880F880F8C73ED
:1038F000B82E48DE10915B035C9A5C9885E08A954F
:10390000F1F7000080915C03823019F081E0809330
:103910005B05D12CB1C08E3409F065C05D9895E28D
:103920009A95F1F700005D9A4C9973CFFE0131969C
:103930009E01235F3F4F83B1482F4270D42E81FDFB
:10394000FACF89B180958F70819380E48A95F1F7E1
:10395000E217F30781F7198190E010FB94F911FB4E
:1039600095F912FB93F913FB92F98C85182F1370BC
:10397000192B83FD10689A8191FD1064282F247003
:10398000C22E82FF02C032E0C32E90FF02C06894B4
:10399000C0F8FB8040E1F49EC0011124FF80F82AAA
:1039A000F0940C8120E1029FC00111240885082BAE
:1039B0000095EE8040E1E49EC0011124EA84E82AEB
:1039C00081E00E94532FB12C10934B05C0924C05FF
:1039D000D0924D05B0925605F0924E0500934F05DA
:1039E000E092520519CF8451823008F049C0CADDF7
:1039F00090915B039F7009F40CCF80915D039F3021
:103A0000E9F5982F9F729032C9F595E19093610581
:103A100010915E0394E0199F90011124422F4C7382
:103A2000B42E90E014FB91F916FB97F9192F90E052
:103A300084FB90F986FB95F9192B90916105D12CA7
:103A40009531B9F490915C0320E090FB26F991FB4D
:103A500023F992FB22F993FB24F9122B482F44708F
:103A6000D42E82FF02C022E0D22E80FF02C06894D2
:103A7000D2F882E00E94532FC12CF1CE94E1C6CF40
:103A8000B12CD12CC12C10E0EACE86EE91E0089545
:103A900008950895E091BB06F091BC060190F08175
:103AA000E02D099510926B0310926A0308958AB96C
:103AB00080958BB98AE68A95F1F700C0089525B103
:103AC000382F3095232325B924B1282B24B9EFE1D1
:103AD000F3E03197F1F700C0000094B1932394B95B
:103AE00090E023B1282391F0892F90E0880F991F4F
:103AF000860F911D67FD9A9597FF02C090E080E0C8
:103B00008F3F910514F08EEF90E008959F5F9E3FE8
:103B100041F78FEF90E0EACF382F23B12095227044
:103B200099B1982B892F80959091310291110DC0F8
:103B300080FB92F981FB93F982FB96F983FB90F964
:103B400085FB95F986FB94F9892F2111832B089524
:103B5000EEEFF1E09081981306C09181DB019C9318
:103B60009281DA019C933396B2E0E133FB0791F73F
:103B70000895EF92FF920F931F93CF93DF9300D09E
:103B8000CDB7DEB77C018B01909168038091310243
:103B9000811118C08FECAE014F5F5F4FBE016E5FA9
:103BA0007F4F8923D5DF8A81F70180838981F801DE
:103BB00080830F900F90DF91CF911F910F91FF9015
:103BC000EF9008958DECE7CF6F927F928F929F9246
:103BD000AF92BF92CF92DF92EF92FF920F931F931B
:103BE000CF93DF9300D000D0CDB7DEB780E88C83D1
:103BF0008B838091610510E0E12C00E08E3009F0AC
:103C000094C014B88FEF85B92AE62A95F1F700C061
:103C100080916E034CDF80916E037EDF809365039D
:103C200080916D0344DF80916D0376DF809366039E
:103C300080916C033CDF80916C036EDF809367039F
:103C400080916F0334DF80916F0366DF8093680398
:103C500080E02DDFBE016D5F7F4FCE01049689DFCE
:103C60002091650300E024FB01F925FB02F9809116
:103C7000660390E084FB90F9092B90E020FB90F91B
:103C800023FB96F926FB93F930E080FB31F983FBA7
:103C900037F986FB34F9932B1091670330E010FB62
:103CA00032F916FB35F9932B30E012FB33F913FB95
:103CB00030F9182F1470132B30E022FB31F9132B3D
:103CC0008C81803819F48B81803831F0802F877097
:103CD00019F0082F10E090E0802F857009F00D7F1B
:103CE000802F877009F0EFC0E02EE92A29F0812F9C
:103CF0008E70E92E09F0E8C0193009F411E0BE0118
:103D00006F5F7F4FCE01029634DF9A818C818917D5
:103D100009F4DCC0809160038C8399818B818917C1
:103D200009F4D7C080915F038B8380916105F12CEA
:103D30008B3009F0D1C005E613E0F12CE12CDD2435
:103D4000D394249A8D2D0E2C01C0880F0A94EAF783
:103D5000AEDE43B189B129B190E0809590959595FB
:103D60008795807130E020953095220F331F220F08
:103D7000331F2074822B942F90959F77892BF80105
:103D800081938F01FFEFEF1AFF0A24E0E216F1049E
:103D9000C1F6539820916503822F8071309166039C
:103DA00000E034FB00F94091670390E044FB91F997
:103DB000092B082B9091680380E094FB87F996FB10
:103DC00085F9082B80E021FB82F923FB85F950E07F
:103DD00031FB51F932FB57F933FB54F9852B50E095
:103DE00041FB50F942FB56F943FB53F9E82EE52A13
:103DF00010E022FB10F980E045FB81F9182BE0E090
:103E000025FBE3F92E2F212B10E035FB12F9122BA5
:103E1000F92FF270FF2E91FF02C030E2F32E93FFD4
:103E200002C06894F4F892FF02C06894F3F895FF1A
:103E300002C06894F2F8E091BB06F091BC060488D9
:103E4000F589E02DDF2CD2942FE0D2228D2D09951B
:103E5000E091BB06F091BC060488F589E02D8D2D1C
:103E600009958111F090560580914E058C83802F25
:103E7000812B61F420E2E21209C080916A039091E3
:103E80006B03019690936B0380936A0380916A039E
:103E900090916B0389389341F8F081E080935B0542
:103EA0000F900F900F900F90DF91CF911F910F9176
:103EB000FF90EF90DF90CF90BF90AF909F908F904A
:103EC0007F906F900895E12C10E019CF80936003EC
:103ED00024CF80935F0329CF809161058B3209F055
:103EE0005FC08AB18F738AB98BB1806C8BB985E65C
:103EF000A82E83E0B82ED12CC12C88248394912C39
:103F000034010C2C01C0660C0A94EAF7862DCFDD33
:103F1000559A5D9A83B199B180958270692A6094AF
:103F20008629F50181935F01FFEFCF1ADF0A24E0B4
:103F3000C216D10429F78091650330E081FB31F985
:103F400084FB32F987FB30F9832FE090660390E021
:103F5000E1FA94F9E4FA95F9E7FA93F9892B1091CB
:103F6000670390E011FB97F917FB96F9E82EE92A11
:103F700080E014FB80F9182F8091680390E081FBAA
:103F800092F984FB93F987FB91F9192B559A5D9867
:103F9000EAE6EA95F1F700C04F9B02C019997DCF80
:103FA00080916105803309F06BC08AB18F738AB943
:103FB0008BB1806C8BB914B88FEF85B9FAE6FA959E
:103FC000F1F700C081E073DD89B1809580936503CE
:103FD00088E06DDD89B180958093660380E467DDBC
:103FE00089B180958093670384E061DD89B1809514
:103FF0008093680380E05BDD82E084B98DEF85B952
:104000002AE62A95F1F700C089B18095809369036B
:104010009091650320E091FB20F910916703012F37
:104020000270022B30E084FB31F985FB32F987FB0B
:1040300030F9832F20916603E0E0E227EF7CE2274E
:1040400027FBE3F98E2B20E014FB27F917FB26F959
:10405000E82EE22AF0E015FBF0F91F2F20E094FB98
:1040600022F995FB23F997FB21F9122B8091680324
:1040700085FFABC06894F5F887FFACC06894F3F88F
:1040800080916105863009F091C04A9B01604C9B8C
:1040900002608091320290913302009709F49FC030
:1040A0000197909333028093320260E084E007DD51
:1040B0008F57990B909362038093610360E080E4D3
:1040C000FEDC8F57990B909364038093630384B154
:1040D000826284B985B1826285B9509A589884B158
:1040E0008B7B84B985B18B7B85B984B1896184B9B7
:1040F000569A2C98F0E4FA95F1F789B1809580935F
:1041000066032C9A289820E42A95F1F789B18095C6
:1041100080936703289A5E9830E43A95F1F789B165
:104120008095809368035E9A2B9880E48A95F1F7D6
:1041300089B18095809365032B9A84B1867E84B97A
:1041400056988091650390E081FB95F983FB94F983
:1041500085FB92F9092B3091660380E031FB80F9F1
:1041600033FB83F935FB86F92091670390E021FB4F
:1041700091F923FB94F925FB97F9892B909168031A
:1041800040E091FB42F993FB45F9E82EE42A10E068
:1041900095FB10F9E0E037FBE1F91E2BF0E027FB7F
:1041A000F2F91F2B20E097FB23F9122BF092560512
:1041B00000934B05E0924C0510934D058C81809344
:1041C0004E058B8180934F056BCE84FF55CF68944D
:1041D000F4F852CF81FF54CF6894F2F851CFE091B8
:1041E000BB06F091BC06C084D184609161036195E7
:1041F00084E065DC62E0F60109958B83E091BB0603
:10420000F091BC06C284D38460916303619580E41D
:1042100056DC62E0F60109958C8359CF80E447DCD7
:1042200089B18D3B09F492C0E091BB06F091BC06C8
:104230000190F081E02D09958FE38AB91BB885E3E1
:104240008A95F1F700008AB18F7C8AB989B1803FE5
:1042500009F47EC0E091BB06F091BC060190F081AC
:10426000E02D0995559A5D988AE08A95F1F700C08E
:1042700089B18F3509F46EC0E091BB06F091BC06A0
:104280000190F081E02D099586E0809361052598E5
:104290002D9A9ADC80E880934E0580934F0580919B
:1042A00063039091640389589F4F8F3E910550F4AA
:1042B000809161039091620389589F4F8F3E9105D1
:1042C00008F44AC0E091BB06F091BC060190F08171
:1042D000E02D099585E38A95F1F7000014B88FEF7A
:1042E00085B98AE68A95F1F700C082E0E0DB89B102
:1042F00080958C7F843329F089B180958C7F8033C1
:1043000089F481E08093310284E080936F0382E03E
:1043100080936E0380E280936D0380E180936C0351
:104320008EE0089580E1C3DB89B180958C7F803F6A
:10433000A9F41092310280E880936F0380E18093AA
:104340006E0380E280936D0380E4E8CF80E30895FC
:104350008BE008958BE2089586E0089580E008954B
:1043600082EF91E0089508950895E091BB06F091E1
:10437000BC060190F081E02D09941092560599B188
:10438000927080917303891751F080917103489B5B
:104390001BC08F5F8093710380E2809356059093DA
:1043A000730399B1987080917203891751F08091CD
:1043B00070034A9B0EC08F5F8093700388E08093E8
:1043C000560590937203089581508093710380E1A4
:1043D000E4CF81508093700384E0F1CF5F985798C9
:1043E00029982198559A5D9A8FE99FE00197F1F7F6
:1043F00000C0000010927403109275035D988EEF58
:1044000090914002992329F09130A1F400C000C09E
:10441000000090917503911103C0199B809375035F
:1044200090917403911103C04F9B8093740381504A
:1044300039F70895923069F795E09A95F1F7E8CF4A
:10444000579A5F988FE891E00197F1F700C000005C
:1044500083B18D3F09F49BC0249A2C9A83B18F3E7F
:1044600009F497C0E091BB06F091BC060190F08181
:10447000E02D09958AB1806C8AB95E985F9A89B1FE
:10448000893B09F488C089B18F3A09F486C08BB1A1
:1044900090EC89278BB9EFE8F1E03197F1F700C094
:1044A000000089B190E0809590958A7199270A97CC
:1044B00009F475C083B1239A2B98EFE8F1E03197A6
:1044C000F1F700C0000085FF0AC083B190E080953D
:1044D000909585FF04C023982B9A81E30895E0917D
:1044E000BB06F091BC060190F081E02D09955E9825
:1044F000569A82E08093400271DF81E0809340020F
:10450000909175039B50809174038B509F3ED8F51A
:104510008F3E08F446C0E091BB06F091BC060190C6
:10452000F081E02D09955E98569A58DF80917503C9
:104530008B508F3EC0F1E091BB06F091BC0601901C
:10454000F081E02D09952998219AF5E3FA95F1F784
:10455000000089B190E08095909588789927892B03
:1045600021F589B190E08095909583709927892BEA
:10457000F1F4E091BB06F091BC060190F081E02DD2
:10458000099580E008958F3E30F68DE3089584E02C
:10459000089588E3089581E008958FE4089582E204
:1045A000089589E208958AE2089588E4089582E4EE
:1045B00008951F93CF93DF935E98569A809161057B
:1045C000803431F08FE99FE00197F1F700C00000DF
:1045D00089B190E080959095880F991F880F991F59
:1045E000D82FDC7380916105883309F0F1C0E09128
:1045F000BB06F091BC060190F081E02D0995249A4C
:104600002C9A8FE891E00197F1F700C0000013B1F8
:10461000109590E010FB94F913FB90F914FB95F9B9
:1046200015FB96F916FB91F9192F99B1909580E039
:1046300095FB82F996FB87F997FB83F9182BC3B199
:10464000C095C27089B1809590E084FB90F9C92B28
:1046500080916105813041F0823231F08F3421F058
:10466000813311F0843059F5E091BB06F091BC061E
:104670000190F081E02D09958AB1806C8AB95E982D
:104680005F9A87EC90E00197F1F700C0000089B1D4
:1046900090E080959095880F991F880F991FD82FCB
:1046A000DC7389B190E08095909534E0959587957D
:1046B0003A95E1F7182F1B70C3B1C095CF76809162
:1046C00061058130E1F0823219F08F3409F093C135
:1046D00055985D9A2198299A29B183B130E02095A7
:1046E000309525FB222720F980958270E091BB064A
:1046F000F091BC060488F589E02D822B09958BB1D9
:1047000090EC89278BB98FE891E00197F1F700C011
:10471000000029B130E02095309583E0359527954C
:104720008A95E1F722703327812F8170822B99B10E
:1047300090959F7041E050E030E020E061E070E053
:10474000941309C0FB01042E02C0EE0FFF1F0A9450
:10475000E2F72E2B3F2B4F5F5F4F4F30510581F714
:1047600090916105923229F081FF03C091E090930E
:10477000610510E033FB12F935FB13F9182BC0E08B
:1047800021FBC5F924FBC1F926FBC4F927FBC3F9BA
:1047900080E030FB80F931FB82F934FB86F936FB8F
:1047A00087F9C82B80E032FB81F990E022FB90F979
:1047B00023FB92F925FB93F9892B10925E05D09388
:1047C000560510934B05C0934C0580934D0551C180
:1047D0008C3031F0982F9F7B19F0863109F04DC055
:1047E000559A85E38A95F1F7000089B123B190E0ED
:1047F0008095909564E0959587956A95E1F78B7023
:1048000030E02095309522703327182F122BB5DD1C
:10481000809171038B3F90F090915E05992371F028
:1048200090E49093610580934E058091700380938E
:104830004F05D091560510925E051DC090916105FF
:10484000903489F311FF03C086E18093610589B13B
:104850008095E091BB06F091BC060488F589E02DB7
:1048600083700995C82F882309F4F2CE8CE08093D9
:104870006105D0915605C0E0EBCE97ED980F9230D0
:1048800018F08D3309F065C010925405109255054B
:10489000A5DD809161058A3229F557985F9A89B123
:1048A00090E08095909595958795959587958470DE
:1048B0009927D82B11E080917403811101C010E079
:1048C00010924002E091BB06F091BC060084F18595
:1048D000E02D62E08091750309958E51880F8093D9
:1048E0005505C9CFE091BB06F091BC060284F38563
:1048F000E02D62E0809174030995809354058091C6
:1049000061058932D1F41D2F12951F7082E08093CA
:10491000400264DD81E080934002E091BB06F091AB
:10492000BC060084F185E02D62E080917503099555
:1049300080935505C0E0DFEF8BCE89B190E0809584
:10494000909544E0959587954A95E1F7182F117059
:1049500092CF883429F0C0E010E0823409F078CE9C
:10496000569A5E9A24982C9AE091BB06F091BC0668
:104970000190F081E02D099595E39A95F1F70000FB
:104980002998219A809161058834C1F489B1809574
:1049900010E082FB11F983FB10F9D9B1D095D595C0
:1049A000D595DC73489B1092510589B1C82FC27010
:1049B00081FD61CF8FEF809351054ACE89B18095FB
:1049C00010E084FB11F985FB10F986FB17F9D9B1CA
:1049D000D095DD0FDD0FDC7389B190E08095909567
:1049E00083709927039709F4106189B18C7009F0DD
:1049F00022CF106220CF813309F04BC0249A2C9A29
:104A000089B18095807F90E4892790E084FB90F9BC
:104A100085FB91F986FB94F910E0C1FB12F9C2FB0A
:104A200015F9C3FB13F9192B24982C9A1C992BC048
:104A30008FE39CE90197F1F700C0000083B19091EA
:104A400076038071892BC9F481E080937603239AE1
:104A50002B9824982C9A8FE891E00197F1F700C0E9
:104A6000000083B1C82FC07285FF10C081E0809321
:104A70005B05DF91CF911F9108951C99E8CF992391
:104A800031F31061E4CF10927603E1CF5E9A80E0BB
:104A900096CE8430E1F7E091BB06F091BC06019020
:104AA000F081E02D0995579A549A5C988FE891E02F
:104AB0000197F1F700C00000C1FD17C01360E0913D
:104AC000BB06F091BC060190F081E02D0995579A44
:104AD0005F988FE891E00197F1F700C0000083B183
:104AE000C82FC27081FFD3CFC1CF4C9BE8CF1260DB
:104AF000E6CF84E392E0089508950895589883E0FE
:104B000091E00197F1F700C00000589A0895509A7B
:104B100058988FED9BE00197F1F700C000000895D1
:104B200058988AE98A95F1F700C0589A87E191E090
:104B30000197F1F700C0000058980895E091BB0676
:104B4000F091BC060190F081E02D09952F9A279AEB
:104B50008FE193E00197F1F700C00000089527E08E
:104B600030E090E040EB4A95F1F7AC01022E02C034
:104B7000559547950A94E2F740FF0CC0589AE3E038
:104B8000F1E03197F1F700C0000058982150310949
:104B900048F70895F0EAFA95F1F7589A4AEB4A95E2
:104BA000F1F700C0F2CF4899FECF85ED8A95F1F775
:104BB000000089B18170489BFECF08951F93CF9369
:104BC000DF93C7E0D0E010E0EEDF0C2E01C0880FCD
:104BD0000A94EAF7182B2197B8F7812FDF91CF912C
:104BE0001F910895CF92DF92EF92FF92CF93C82F3B
:104BF0008EDF96DF8C2F8C63B2DF80DF509888EEDB
:104C000093E0489920C0489BFECF4899FECFD6DF5D
:104C100090E0B0E0A0E0CC24D82EE92EFA2ECEDF32
:104C2000C82AC11108C0CADFC82FC8DF7601DD2439
:104C3000CC24C82ADC2AC701B601CF91FF90EF909F
:104C4000DF90CF9008950197E1F6C12CD12C760129
:104C5000F2CF8F929F92AF92BF92CF92DF92EF925C
:104C6000FF92CF93C1E0C093600583E0BBDF672B69
:104C7000682B692B61F4C0935B05CF91FF90EF9097
:104C8000DF90CF90BF90AF909F908F90089580E07D
:104C9000A9DF611571058105910509F454C0892EBC
:104CA0009924AA24BB246C01EE24FF24272F2095ED
:104CB000609580E887FE80ECC7FC8F7780934B057A
:104CC000882D8F779C2D9F7786FC8068C6FC906826
:104CD00030917803930F9093780330917703830F8B
:104CE0008093770390934E0580934F0580E022FBDD
:104CF00082F923FB84F924FB85F925FB83F9809352
:104D0000560580E020FB83F921FB82F926FB80F920
:104D100027FB81F9282F80914B05282B60FD11C0BE
:104D200020934B0561FF05C080914D058460809301
:104D30004D0562FFA2CF80914B05806280934B05A9
:104D40009CCF2061EDCFC0935C0597CF89B18C3F9C
:104D500011F480E00895DBDEE3DE8BE300DFCEDEDE
:104D60008FE193E00197F1F700C00000D9DE83E600
:104D7000F6DE86E4F4DEC2DE5098589A83E032DF35
:104D8000672B682B692B29F38AE0089581E492E070
:104D9000089508950895982F9770906490937C00DB
:104DA00090917A00906490937A0090917A0096FDA9
:104DB000FCCF90917A00906490937A0090917A0061
:104DC00096FDFCCF2091780030917900482F50E07B
:104DD00080917903440F551F882339F0C901465843
:104DE0005C4FFA01318320830895C90180589F4F99
:104DF00046585C4FFA0120813181821B930B97FF4B
:104E000002C090E080E08F3F910519F014F08FEF21
:104E100090E00895E091BB06F091BC060190F0810E
:104E2000E02D099581E0809379030895FF920F9317
:104E30001F93CF93DF931BB885E38A95F1F70000AA
:104E400089B18095982F9F7DC1E0983019F080320C
:104E500009F0C0E08FEF8BB9579A5F988FE891E027
:104E60000197F1F700C0000083B18D3E41F4C0E02E
:104E70008C2FDF91CF911F910F91FF90089587E8BC
:104E800080937A0083B18AB1806C8AB95E985F9A08
:104E90008FE99FE00197F1F700C00000F3B024987C
:104EA000249AD4E08D2F77DF080F111DDF5FD830F3
:104EB000C9F79DEFF9120AC0055C1940073E13407F
:104EC000B0F68BB18C608BB9C5E0D2CF83B1809541
:104ED0008093620583B18E3F11F0CC2339F08BB102
:104EE000837C8BB9509A5898CEE2C2CF10927A0048
:104EF000BFCF1F93CF93DF9384E04DDFD82F85E0A2
:104F00004ADFC82F86E047DF182F87E044DF109282
:104F1000790390916105953099F4D0934E05C09531
:104F2000C0934F0589B180958F7080934B05199B75
:104F300023C081E080935B05DF91CF911F9108959D
:104F40009E32D1F4C095C0934E05809580934F0555
:104F5000D095D093510510951093520583B19FE7DA
:104F6000892790E080FB90F981FB92F985FB91F90C
:104F700087FB93F990934B0510925F05DDCF8DE48D
:104F800092E00895509858980895EF92FF920F93E9
:104F90001F93CF93DF937C01C62FE6E1F5E082E219
:104FA000DF011D928A95E9F7E091BB06F091BC06FE
:104FB00000A4F1A5E02D09950091940010919500B1
:104FC000D0919000B0919100A09171001092950045
:104FD0001092940081E08093910010929000589A72
:104FE000509A809194009091950020918A03820FAD
:104FF000911DF701B7016C0F711DE617F70791F5C9
:10500000589825E02A95F1F70000589A5098109288
:10501000910010926F001093950000939400D0932C
:105020009000B0939100A0937100C0E080E820E070
:1050300039B1932F917030FD33C0A8E0AA95F1F7F4
:10504000489B07C0EC2FF0E0EA5EFA4F2081282B46
:105050002083869511F4CF5F80E84899E8CF91507E
:10506000E1F721C0319128E0589837FF08C00000CF
:10507000000000000000000000000000589A40916D
:10508000940050919500481B590B57FDF8CF589A42
:10509000330F40918A03840F911D215029F7ADCF22
:1050A000215009F0C5CFE091BB06F091BC0602A4E7
:1050B000F3A5E02D0995B0EABA95F1F78C2FDF91B1
:1050C000CF911F910F91FF90EF900895CF93DF93B1
:1050D000D09196056091B90686E995E056DFC82F14
:1050E000D23039F4813229F010929605DF91CF91B8
:1050F00008954C2F50E066E175E087E995E00E9445
:105100000A3AC0939605E6E1F5E082E2DF011D92DE
:105110008A95E9F7EBCFCF93DF930F92CDB7DEB748
:1051200080E480938A0319822FEF85EA9EE0215064
:1051300080409040E1F700C0000061E0CE010196A0
:1051400024DF833081F48091160510925F0585304D
:1051500061F098E490938A03883049F089E00F90D9
:10516000DF91CF91089580E0FACF83E1F8CF82E11B
:10517000F6CF8CE0EDEEF2E0ABE4B5E001900D92FD
:105180008A95E1F710925C0580918A04882341F0AA
:105190001092540510925505109253051092500527
:1051A0000895669B0AC0AFE9B4E084E1EDEAF4E05B
:1051B00001900D928A95E1F70895ABE8B4E0F5CF40
:1051C00084E1669909C0EBE8F4E0ADEAB4E001904F
:1051D0000D928A95E1F70895EFE9F4E0F6CF80911A
:1051E000C104882369F081E080935A05E0919A0612
:1051F000F0919B060280F381E02D099510925A05EB
:1052000008958CE0E0EAF4E0ABE4B5E001900D92A3
:105210008A95E1F70895CF92DF92EF92FF920F9374
:105220001F93CF937C016B018A01C0E08C2F90E02B
:105230008017910740F0CF911F910F91FF90EF9051
:10524000DF90CF900895F601E80FF91F60818E0D71
:105250009F1D0E94223ACF5FE9CFCF93C82F81E1F3
:1052600090E00E941A3A80939806C0938A04E091D5
:10527000BB06F091BC060484F585E02D81E009951C
:1052800080918A04811108C00E946006789481E0B0
:1052900080935F05CF916DCF8091D700816080931F
:1052A000D700F4CF2CB19091560531E026FB222790
:1052B00020F9231709F46EC0831709F46BC084E149
:1052C000EBE8F4E0DF01282F1D922A95E9F780939F
:1052D0008C0496959695292F2F7090914B05892FC8
:1052E000829530E038273F70382782FB30F983FB06
:1052F00031F930938E0480E094FB85F995FB84F9B5
:1053000030914C05822B932F907C892B80938D04B8
:1053100090914D05943019F4806C80938D04909198
:10532000500580915305903869F5803861F530FF5C
:1053300003C08FEF80938F048FEF31FD28C08091E1
:105340004E058058990B109291048093920480919D
:105350004F0580958058990B109293048093940484
:10536000809151058058990B109295048093960472
:105370008091520580958058990B109297048093E4
:1053800098040895911190938F048823C1F280931B
:105390009004D5CF81E080939F048BE0EBE4F5E0AF
:1053A000A0EAB4E001900D928A95E1F7E5EEF2E013
:1053B0002FEF80E03191391301C0282F8F5F8830A3
:1053C000C9F72093AB040895C09B2FC081E088BB30
:1053D000809148058F5F80934805909148058091A2
:1053E0004705981710F1109291001092710080916A
:1053F0003905843059F4E0919A06F0919B060084B7
:10540000F185E02D70E060E080E00995809139053C
:10541000853059F4E0919A06F0919B060284F38559
:10542000E02D70E060E080E0099408950F931F93F1
:10543000CF93DF93C1E9D0E01882E1E7F0E010827A
:10544000609339059C01A8EEB3E00E94FB39DC01B2
:10545000CB0122E0B695A795979587952A95D1F728
:105460008C019D01015011092F4F3F4F89012227C7
:105470003327009347051092480566277727681B56
:10548000790B70939500609394001092900083E0E4
:10549000888381E088BB1082DF91CF911F910F91AB
:1054A000089581E0809378050895E2EEF0E0808130
:1054B000846080830895089542E361EC81E00E9456
:1054C000840542E260EC82E00C948405EF92FF9246
:1054D0000F931F93CF93DF93CDB7DEB7CF5FD10983
:1054E0000FB6F894DEBF0FBECDBF10910F05F09040
:1054F0001005812F90910E05913089F0993009F4B3
:1055000047C1C150DF4F0FB6F894DEBF0FBECDBF0D
:10551000DF91CF911F910F91FF90EF90089590919F
:105520000D05913A09F034C19091E800977F90936E
:10553000E80023E0F21221C11230E1F490913C0521
:105540002FEF290F243020F4892F923009F081E0C9
:1055500022E029839A838B838AE08C8364E070E065
:10556000CE0101960E9421048091E8008B77809300
:10557000E800C7CF133059F419838FEF9FEF9B8357
:105580008A8384E08C831D8365E070E0E9CF4091DD
:10559000980640938B031531C1F48DE090E0909311
:1055A0003B0580933A05EDE9F6E0ACE8B3E089EA23
:1055B00096E021912D938E179F07D9F760913A05B8
:1055C00070913B058BE893E0CDCF1831C9F481ECA5
:1055D00090E090933B0580933A052CE8E22E23E07F
:1055E000F22E00EA10E0C8010E941A3AD7018D930A
:1055F0007D010F5F1F4F0036B1E01B07A1F7DECF23
:10560000103181F48DE090E090933B0580933A0552
:105610008CE0EBE4F5E0ACE8B3E001900D928A9504
:10562000E1F7CCCF163179F58091960590E09C0199
:105630002D5F3F4F30933B0520933A0520917D0528
:1056400020938C03209138052130D1F010928D03E6
:1056500083E090E090933B0580933A05AFCFF9014A
:10566000E557FC4F2C563A4FD9012C9120834F5FC0
:10567000242F30E08217930794F710927D059ECF78
:1056800042E00296F5CF1731C1F480E390E09093A9
:105690003B0580933A059BE8E92E93E0F92E00E163
:1056A00010E0C8010E941A3AF70181937F010F5F51
:1056B0001F4F00341105A9F781CF1931C9F481E8D2
:1056C00090E090933B0580933A058CE8E82E83E0C8
:1056D000F82E0CEA11E0C8010E941A3AD7018D9306
:1056E0007D010F5F1F4F0C32B2E01B07A1F766CFA1
:1056F000113109F039CF85E090E090933B0580931C
:105700003A058091610580938B0360915B058091E0
:10571000B20650E0811154E09091AA06E8E09E9F05
:10572000C00111242091A906F0E12F9F90011124BE
:10573000822B862B2091AC0670E2279F90011124CA
:10574000822B2091AB0690E4299F90011124822B9B
:1057500020915F05A0E82A9F90011124822B852BC0
:1057600080938C038091BA0680938D0340938E03BF
:105770008091770580938F0321CFB1E0FB12F4CEA7
:10578000113009F0F1CE6EE070E08FE994E0EACEDE
:1057900080910D05813209F0B4CE609113057091AE
:1057A00014058091E800877F8093E800E3E0FE1213
:1057B00009C0CE0101960E947F041F3039F48A810E
:1057C00080933C058091E8008E77D1CE0A81053226
:1057D00009F4AAC18CEF800F823008F493C1E091E4
:1057E0009A06F0919B060284F385E02D6AE070E052
:1057F0008FEF0995123109F05AC1003289F48D8179
:10580000885F809363058E81885F809379058F819F
:10581000885F80939C068885885F80937605D2CFC9
:10582000013009F0A6C08D818F3F09F08DC08E81B7
:105830008130A9F56091A90684E190E00E94223AA6
:105840006091AC0685E190E00E94223A6091AB063F
:1058500086E190E00E94223A6091AA0687E190E0FA
:105860000E94223A6091630568508CE190E00E94AA
:10587000223A6091790568508DE190E00E94223AC9
:1058800060919C0668508EE190E00E94223A6091FF
:10589000760568508FE190E00E94223A93CF8230E3
:1058A00009F090CFE091BB06F091BC0606A0F7A1ED
:1058B000E02D09958FEF8093B2066FEF8CE390E0B7
:1058C0000E94223A81E08093B70661E08BE390E08A
:1058D0000E94223A10925E0560E08DE390E00E9403
:1058E000223AEEE7F5E080E08F5F81938831E1F7BF
:1058F00048E150E06EE775E081E290E08CDC61E029
:1059000080E290E00E94223A0CEA10E064E5600F29
:10591000C8010E94223A0F5F1F4F0B3AF1E01F07A8
:10592000A9F70CEA11E06FEFC8010E94223A0F5F5D
:105930001F4F0C3222E01207B1F78FE08093B606BA
:105940006FE08BE190E0A8CF83FB992790F99093CB
:10595000AA0684FB992790F99093A90685FB9927BD
:1059600090F99093AC0686FB882780F98093AB066C
:1059700029CF033051F46D81862F90E09093AF06CC
:105980008093AE0689E190E087CF063021F46D81E7
:105990006093B606D6CF003839F460914B0560931A
:1059A000AD0688E190E078CF003451F46D816093CA
:1059B0007A058E81882309F405CF83E190E06CCFCE
:1059C000003149F4E091BB06F091BC0602A0F3A1BE
:1059D000E02D0995F7CE083071F46D8181E190E0FA
:1059E0000E94223A8E81882309F4ECCE75E07A95E4
:1059F000F1F70000E7CF023009F0E4CE8E8190E0AD
:105A00006D81CB960E94223ADDCF823081F48E8167
:105A10006F817885E0919A06F0919B06043049F4F5
:105A20000084F185E02D0995CDCE8FEF7AC080E01E
:105A300078C00284F385E02DF6CF82E080933805AC
:105A40008D818093B9069E8190937D059F8190936F
:105A50009605988590939705833010F4F092380559
:105A60001092490510917D05113009F0ABCE80915F
:105A70003805833009F0A6CEE0919A06F0919B0696
:105A80000480F581E02D0995109338059BCE12E036
:105A90005FC03D9131932F5F62C0833009F072C0C7
:105AA00040E850E066E975E08CEA91E06AC01431A4
:105AB00061F440EC50E0BE016B5F7F4F80EA90E004
:105AC000AADB81E080937B057DCE133109F07ACE8D
:105AD000DE011596EEE7F5E086E995E02D9121933C
:105AE0008E179F07D9F78D8D6FEF813041F448E114
:105AF00050E06EE775E081E290E08DDB61E080E2EE
:105B000090E0CACE123199F68D8170E060E0882372
:105B100009F480CF813009F078CF8E81882309F491
:105B200084CF6FEF70E076CF123109F0C0CF8B8158
:105B3000882309F482CF182F95E08F3F49F4109104
:105B400049059091B906911B112309F4A0CF1B5F61
:105B5000DE011496E12FF0E0EA56FA4F20E0291317
:105B600098CF8F3F79F480917D0593E0909338052D
:105B7000823009F092CF4FEF50E066E975E08CEA91
:105B800090E049DB109349056DCFCF9380918A0453
:105B90008111A5C080910C05843009F0A0C081E07E
:105BA0008093E9008091E80080FF11C0669B4CC0A3
:105BB0006EE070E0669B4BC08FE994E050E040E0FF
:105BC0000E9485038091E8008E778093E80082E050
:105BD0008093E9008091E80082FF81C08091E80015
:105BE00085FF78C0669936C09091F1008091F100F0
:105BF0008091F1008091F100C091F10091116AC093
:105C000061E070E0811102C070E060E07195619523
:105C10007109E0919A06F0919B060084F185E02DD0
:105C2000099561E070E0C11102C070E060E071951B
:105C300061957109E0919A06F0919B060284F385C3
:105C4000E02D8C2F099546C060E270E0B3CF8BE861
:105C500094E0B4CF8091F3004091F200582F70E0AF
:105C600060E082EC94E00E94133A8091F30060912E
:105C7000F200782F50E040E082EC94E00E94D303E1
:105C80008111F3CF8091C2048C30D1F48091C30490
:105C9000833001F5E0919A06F0919B060284F3852A
:105CA000E02D70E060E080E00995E0919A06F091C7
:105CB0009B060084F185E02D70E060E080E0C2CFBB
:105CC000843079F48091C304823020F08091C40440
:105CD000809346058091E8008B778093E800CF9110
:105CE0000895813049F48091C5049091C604909341
:105CF0003F0580933E05EECF853079F48091C30453
:105D0000813041F78091C4049091C50481509F4F28
:105D10009595879580934205DDCF8A30D9F680919D
:105D2000C3048130D9F4E0919A06F0919B06008477
:105D3000F185E02D8091C404833049F470E060E087
:105D400080E009958091C40480934A05C3CF609197
:105D50003E0570913F0580914205F3CF835082301C
:105D600008F0B8CFE0919A06F0919B060284F38583
:105D7000E02D8091C404833009F49ECF60913E05EC
:105D800070913F05809146055DCFCF93DF93D82F6B
:105D9000C0E0CD1303C0DF91CF910895F6DE0E94DD
:105DA000B2088FE99FE00197F1F700C00000CF5FD4
:105DB000F0CFEF92FF920F931F93CF93DF93CDB766
:105DC000DEB766970FB6F894DEBF0FBECDBF81E099
:105DD0008093C1040E94D30F9A8389830E94EB0EA3
:105DE0009C838B830E9467199E838D830E94A60BE0
:105DF00098878F830E94B51A9A8789870E94451DCC
:105E00009C878B870E94B0219E878D870E94C62623
:105E1000988B8F870E94B5139A8B898BB0D89C8BF7
:105E20008B8B0E9479259E8B8D8B8E010F5F1F4F70
:105E30007E0187E1E80EF11C0E94B208D801ED91C5
:105E4000FD918D01F0939B06E0939A060190F081FD
:105E5000E02D0995E0919A06F0919B060680F78166
:105E6000E02D099580936105811114C00E151F0561
:105E700019F78AEF8ADF8091610566960FB6F8946C
:105E8000DEBF0FBECDBFDF91CF911F910F91FF906D
:105E9000EF900895833169F70E94CB1090939B0691
:105EA00080939A06E6CF0F931F93CF9398E0899F34
:105EB00080011124C0E0C017110624F0CF911F917A
:105EC0000F91089562DE0E94B20883EF91E001977E
:105ED000F1F700C00000CF5FEECF57DE0C94B208A0
:105EE00089E592E00895F9011082692F77276330E0
:105EF0007105F1F158F461307105D1F0623071052E
:105F000059F190E080E030E020E00EC089E090E0C0
:105F10002EE031E06132710539F08DEB93E025E23E
:105F200031E06232710569F7FA0131832083089507
:105F3000669B3FC082E0808320919806822F90E08C
:105F4000935F9093A3028093A2022093A80282E120
:105F500090E028E932E0E8CF669B07C02CEF30E004
:105F6000669B2CC089E290E0DFCF22EE34E0F8CFD0
:105F7000992781309105D1F0009791F0029709F6A9
:105F800082E080838091980690E08D9690939502B0
:105F90008093940280916C0290E02CE632E0C4CFB2
:105FA000E8EFF0E0849190E09F01BECFE2EEF0E0F8
:105FB000F9CF82E190E022E135E0B6CF80E390E0D6
:105FC000B3CFC2D79093BC068093BB06DC01149676
:105FD000ED91FC910995E091BB06F091BC0606801D
:105FE000F781E02D0995C4E0C093BA0664E080E132
:105FF00090E00E94223A86E58093770566E582E18B
:1060000090E00E94223A66E08AE190E00E94223A03
:1060100081E190E00E941A3A9CEF980F943008F0CA
:10602000ACC0809398060E94B51A90939B0680930B
:106030009A06DC01ED91FC91099552DF9093E504FD
:106040008093E4040E94F8399093E3048093E2047F
:10605000DC01ED91FC9109958093E6049CB1E091FF
:10606000E404F091E50496FB992790F921E092274A
:10607000928B0484F585E02D0995E091E404F0917C
:10608000E5040088F189E02D099502E010E0D5E0F3
:10609000EE24E394F12CDD24DA94E091BB06F09138
:1060A000BC060484F585E02D81E00995E091E404C7
:1060B000F091E5040680F781E02D09958CB1E0911F
:1060C000E404F091E50486FB882780F991E08927B4
:1060D0009289981741F0E091BB06F091BC0602A0AE
:1060E000F3A1E02D0995629B02C01A9915C0BFEF7C
:1060F00021EE84E0B15020408040E1F700C0000074
:10610000629B02C01A9908C0E091BB06F091BC06E0
:1061100004A0F5A1E02D099580915B05882309F481
:10612000AEC08091AA068111AAC0E091BB06F09191
:10613000BC060484F585E02D09958091AA02882388
:1061400021F11092AA028091AB06811105C08091C5
:106150004B05806280934B05E091BB06F091BC0635
:106160000680F781E02D0995E091BB06F091BC0611
:106170000280F381E02D099533C0C093980664E056
:1061800081E190E00E94223A4ECFE091E404F09148
:10619000E5040088F189E02D0995882309F1E09153
:1061A0009A06F0919B060190F081E02D0995C0912F
:1061B0006105E0919A06F0919B060680F781E02D3B
:1061C00009958C130DC010924B0510925B0581E070
:1061D0008093AA02AFE9BFE01197F1F700C0000079
:1061E00081E09091E604911101C080E0E091E40427
:1061F000F091E5040190F081E02D099580917405FE
:10620000909175058E3F910509F06FC016BCD5BD04
:10621000E091E404F091E5040480F581E02D099516
:10622000F0927505E092740580915C05811165C05E
:10623000E091E404F091E5040480F581E02D0995F6
:10624000E091E404F091E5048091E604882309F4E8
:1062500074C080915B058111D09261050684F78539
:10626000E02D0995E091E204F091E3040280F381CE
:10627000E02D0995882309F410CFA895F3CFA4D871
:10628000E091E404F091E5040084F185E02D0995A6
:106290008091B706823088F480916005811116C024
:1062A000809161058C3109F49BCFE091BB06F091A0
:1062B000BC060684F785E02D5ECFC1E081E0F3DD0A
:1062C000CF5F8091B706C817C8F3E6CF8091E60488
:1062D0008111E6CF10927805B5E0BA95F1F700008C
:1062E000809178058823C1F3DBCF81309105B9F423
:1062F000A8990BC081E080935C05E091E404F091E3
:10630000E5040280F381E02D9ACFA89B8DCFA89A57
:1063100016BC1093750500937405D5BD85CF029703
:1063200009F082CFA89BE6CFA89B7ECFA89A15BC88
:10633000109275051092740577CF0284F385E02DD5
:106340000995ABCEE2EEF0E080818093E704108205
:1063500008958091E7048093E200089514B88FEFC8
:1063600085B91AB88BB910BA11BA089510929B0664
:1063700010929A06EBE4F5E081E0848B138A109288
:10638000EF04E9EAF6E01186148613861286089572
:106390008330D1F49091D7029F3FB1F491E0909374
:1063A000E804109256052091D702281771F19091B8
:1063B000E904223079F4833031F59B5F9093E9044E
:1063C00090E29093560521C09091E8049111E9CF95
:1063D000892F0895233049F4813079F38230A9F46C
:1063E00095509093E90490E1ECCF213029F4882373
:1063F00021F3833051F4F4CF211107C08230E9F248
:10640000813019F4EDCF882359F39091E9049093EA
:106410004E058093D70291E0DBCF982F8091EB045B
:10642000482F491B550B9A0157FF03C03195219501
:106430003109621718F49093EB04892F0895982F6F
:106440008091EA04482F491B550B9A0157FF03C05E
:10645000319521953109621718F49093EA04892F38
:10646000089514BEF894A8950FB6F894A895909145
:106470006000986190936000109260000FBE8823C6
:1064800059F088E19FE00FB6F894A89580936000DA
:106490000FBE90936000789408958091ED0481116F
:1064A00025C02091AE063091AF064AE0429FC00160
:1064B000439F900D11242091840030918500821714
:1064C000930798F410928500109284008091ED0457
:1064D00081508E3F18F48EEF8093ED0481E090910F
:1064E000F004911180E08093F004089588EA91E629
:1064F000E2CF90914B05892F8F7C79F195FF19C0E0
:1065000080914C0520914D05822B292F2071822BE3
:1065100079F481E08093F1048091EF04882341F0C5
:106520002091F004211104C08095892380934B05AC
:1065300008958091F104813079F72091EF04109251
:10654000F1048091EE048F5F8093EE04292730E000
:106550003093B1062093B006DFCF9111DDCF80914B
:10656000EE048823C9F224E630E0853021F084303F
:1065700049F429E130E03093AF062093AE06109243
:10658000EE04CACF8330D9F78091B0068093EF0430
:10659000F6CF80914B05803D09F43FC0803EE9F184
:1065A00081111EC01092ED0480E09091ED049E3F99
:1065B00009F06AC09FEF9093ED04813081F59091CE
:1065C000A906911180E08093A906E0919A06F091C6
:1065D0009B060284F385E02D68EC70E084EF09945B
:1065E000803C61F480915605843031F0883021F090
:1065F000803211F08031B1F682E003C085FFD2CF46
:1066000083E09091ED049111D0CF1092850010920B
:10661000840091E09093ED04C8CF81E0F2CF823006
:1066200061F59091A9069923B9F080914F058111E8
:1066300004C084E08093B206C8CF8F3F11F488E095
:10664000F9CF80914E05811102C080E1F3CF8F3FD9
:1066500009F0BBCF80E2EECF90915605943019F44B
:106660001092B206B2CF983021F3903111F486E047
:10667000E1CF903209F0A9CFDDCF833009F0A5CF6B
:1066800081E08093F204A1CF0895CF93DF9300D0EF
:10669000CDB7DEB7B091B306B983A091B406AA8393
:1066A00020914B05FE013196AE014D5F5F4F819108
:1066B000982F922381F0382F31953823982F931BF0
:1066C000982380958223632F622309F0892B292345
:1066D00069F1232F282B4E175F0749F720934B05AD
:1066E0003091B506332309F44AC0822F90E0FC01B3
:1066F000F595E7953230E1F0BC0175956795759594
:106700006795333049F14E2F4470313009F067C03E
:10671000FC01EE0FFF1FE270880F991F880F991F71
:1067200088708E2B6170862B842B24C0282FD3CFAA
:10673000AC01F3E0440F551FFA95E1F74870BC0136
:10674000660F771F962F9470942B4E2F4270492B13
:1067500023FB882780F9E8CFAC01440F551F440F75
:10676000551F4470E1704E2B880F991F8870842B41
:106770006270862B422F407F842B80934B05809143
:10678000F204882339F11092F2042F7D50E040E0AA
:1067900080E0E22FF0E0BF01042E02C075956795FE
:1067A0000A94E2F76170860F4F5F5F4F48305105E2
:1067B00091F7811120C08091AD06882359F0809314
:1067C0004B0581E08093EC048EEF90E0909375058B
:1067D000809374050F900F90DF91CF91089553E04F
:1067E000880F991F5A95E1F788706170862B922F58
:1067F0009270892B99CF813051F490914B05903351
:1068000049F794E090934D0510924B05DBCF84300F
:1068100049F43F5F343019F03093B506DBCF109266
:10682000B506D8CF8230B1F6B21303C01092B306CA
:10683000D1CFA21303C01092B406CCCFB11103C0C4
:106840002093B306C7CFA111C5CF2093B406C2CF02
:10685000CF93DF9300D000D000D0CDB7DEB78091CA
:106860004B058C8380914C058D8380914D058E83E3
:1068700019821A821B82AEE7B5E090E041E050E059
:106880008D91882359F1E92FE695E695E69524E068
:1068900030E02C0F3D1F2E0F311DF901208130E01B
:1068A000692F677002C0359527956A95E2F720FF3A
:1068B00015C08150E82FE695E695E69521E030E099
:1068C0002C0F3D1F2E0F311DF90187709A0101C059
:1068D000220F8A95EAF78081822B80839F5F98310F
:1068E00079F6898180934B058A8180934C058B8151
:1068F00080934D0526960FB6F894DEBF0FBECDBF30
:10690000DF91CF9108958091A9068823A9F0809105
:10691000560582FD10924F0583FF03C09FEF9093B1
:106920004F0584FD10924E0585FF03C08FEF8093C5
:106930004E058FEF80935605809161058234E9F012
:106940008431D9F0809156058F3FB9F0982F90731C
:10695000903319F08C708C3081F481E080935E0567
:106960008091560524E0829FC0011124807F909180
:106970004D05892B80934D0504C080915E058111E2
:10698000EFCF0895AF92BF92CF92DF92EF92FF9236
:106990000F931F93CF93DF93C0914B058091B20665
:1069A000823049F170F4882309F467C0DF91CF91F8
:1069B0001F910F91FF90EF90DF90CF90BF90AF901D
:1069C0000895843009F4DFC0863081F79091610525
:1069D000963309F071C00C2E00FAC1F901FAC7F91B
:1069E00002FAC3F903FAC6F906FAC2F907FAC0F9BE
:1069F000C0934B05DBCF80914C05D82FF0906105FB
:106A00000CEA11E0C80116D5A801485F5F4F6A0182
:106A10008F3F09F4CEC0F812CCC00F5F1F4F7E012C
:106A2000AA24A394B12CC80105D58F3FE1F0982F7B
:106A300092959F70950102C0220F331F9A95E2F73D
:106A4000AE0142235323452B71F08F70A50102C084
:106A5000440F551F8A95E2F7CA01E42AF92A2095C6
:106A60003095E222F3220F5F1F4FC016D106D9F6F0
:106A7000F0924C05E0924B0599CF809161058333EC
:106A800009F094CF809152058093500580914E0576
:106A90008093530580914F05809354058091510553
:106AA00080934E051092550580E8809351058093A0
:106AB000520580934F057ACF492F477F392F3B7F6F
:106AC00081E09A3009F080E021E09F3209F020E077
:106AD000822B21E09E3309F020E0822B21E09D31C2
:106AE00009F020E0822B21E09F3709F020E0822B83
:106AF00021E0993709F020E0822B21E0913309F061
:106B000020E0822B21E0403109F020E0822B21E0BF
:106B10003B3109F020E0822B51E0292F2F7E2332D8
:106B200009F050E0852B21E0413409F020E0822B70
:106B300011F4333761F40C2E00FAC1F901FAC7F9E8
:106B400002FAC0F906FAC2F907FAC6F951CF99302C
:106B500011F0923151F40C2E02FAC3F903FAC7F97D
:106B600006FAC2F907FAC6F943CF933109F01ECFEE
:106B70000C2E00FAC2F901FAC0F902FAC3F903FABD
:106B8000C1F9C0934B0590914B0580914C05292F7D
:106B90002F7330E4839FA0011124242B20934B05F5
:106BA0008C7F9295969596959370892B80934C0542
:106BB000FDCE86015CE2C51652E0D50609F022CF73
:106BC0007E0156CF0F931F93CF93DF930BE415E015
:106BD000D0E0C0E0C230D10541F0F801838190E0FF
:106BE00084559F4F27D4F801838321960F5F1F4F51
:106BF000C530D10579F7DF91CF911F910F9108959D
:106C00008091AA06811110925B0580914E058759EB
:106C10008F3440F08091550590915405892B8F77E2
:106C200009F445C010925F058091AC06811107C040
:106C30008091AE069091AF06892B09F05ADC63DE95
:106C4000A8DC8091AC06811101C09CDE01DE809140
:106C5000AC06811101C019DD8091B60680FF04C029
:106C600090916105933191F081FF04C0909161058D
:106C70009D3061F082FF04C090916105993031F040
:106C800083FF05C080916105863009F49BDF05DC38
:106C90009091EC049923F1F080914B0585FF16C08B
:106CA0008F7D80934B0582E08093EC040895809162
:106CB0005F05882309F4B8CF80E880934F0580935F
:106CC0004E058093510580935205AECF923011F45A
:106CD0001092EC0408951F93CF93DF9310927A05DE
:106CE00060E083E190E0AED3C9EAD6E0188260E0CC
:106CF00084E190E0A7D31B8260E085E190E0A2D31D
:106D000089E190E09E838D8369E19CD31FE01D871C
:106D10006FE08BE190E096D31A8260E086E190E02C
:106D200091D3198260E087E190E08CD31C8260E00F
:106D300088E190E087D381E08E8761E08BE390E08B
:106D400081D310925E0560E08DE390E07BD368E034
:106D50008CE190E077D380E18093630567E08DE17B
:106D600090E070D3109379056BE08EE190E06AD3E8
:106D700083E180939C066CE08FE190E063D384E133
:106D800080937605DF91CF911F9108950F931F9304
:106D9000CF93DF938CEA90E04DD38F3F59F4CCEA48
:106DA000D0E06C2F6C5ACE014DD32196CB3A81E0C6
:106DB000D807B9F780E290E03DD38F3F91F4C1E26C
:106DC000D0E06C2F6152CE013DD32196C534D10560
:106DD000C1F7EEE7F5E080E08F5F81938831E1F75E
:106DE0000FC08130B1F70EE715E0C1E2D0E0CE016F
:106DF00021D3F80181938F012196C933D105B9F7C9
:106E000084E190E017D38F3F29F4DF91CF911F9158
:106E10000F9161CF83E190E00DD380937A0584E1F7
:106E200090E008D38093A90685E190E003D3809396
:106E3000AC0689E190E09093AF068093AE068BE1BB
:106E400090E0F8D28093B60686E190E0F3D280938A
:106E5000AB0687E190E0EED28093AA0688E190E04D
:106E6000E9D28093AD068BE390E0E4D28093B7063D
:106E70008DE390E0DFD280935E058CE390E0DAD280
:106E80008F3F11F08093B2068CE190E0D3D2885FFF
:106E9000809363058DE190E0CDD2885F8093790582
:106EA0008EE190E0C7D2885F80939C068FE190E0EE
:106EB000C1D2885F80937605DF91CF911F910F91AA
:106EC00008950E940806F894FFCF0E940806F894DF
:106ED0000FB6F894A8958091600088618093600057
:106EE000109260000FBEF0E0E0E00995729A6A9897
:106EF00087B18F7387B988B18F7388B9E1E6F0E005
:106F000080E88083108210BA11BA28DA769A6E98D7
:106F10008FE99FE00197F1F700C00000E091BB0608
:106F2000F091BC060484F585E02D80E009959FEF83
:106F300025EA8EE0915020408040E1F700C000003B
:106F400085E08093810008958BEA92E008952AE11C
:106F50002A95F1F700C098B1906C98B995E09A9590
:106F6000F1F70000000098B19F7398B927E02A95C7
:106F7000F1F746EF54E0FA0198E0479A29E02A95A4
:106F8000F1F700000000208120FD1DC028E02A95B7
:106F9000F1F700C020812695208300C0915069F749
:106FA000479A94E09A95F1F700C0479823E02A9514
:106FB000F1F7000031969E2F941B9817E8F288B1E4
:106FC000806C88B90895479827E02A95F1F7E2CFB9
:106FD00088B1806C88B982E395E09A95F1F700005A
:106FE00096B1907C903C31F08150B1F798B19F738D
:106FF00098B908959AE19A95F1F700C096B1907CFE
:10700000903C91F781E00895CF9387B18F7387B952
:1070100088B1806C88B930E13A95F1F700C086B14B
:10702000807CCFEF803C09F0CFC03799FECF85E15F
:107030008A95F1F7000088E0CFEFC695379BC068CE
:107040000000000095E19A95F1F78150B1F787B102
:10705000806C87B988B18F7388B92091060530910B
:1070600007052115310509F48BC080910505823093
:1070700059F5C3FF1DC081E08093AA06C4FF1BC061
:1070800081E08093A906C5FF19C081E08093AC061A
:10709000C6FF17C081E08093AB06809106059091F2
:1070A000070501979093070580930605C1E08CC002
:1070B0001092AA06E3CF1092A906E5CF1092AC0673
:1070C000E7CF1092AB06E9CF843041F4213031058F
:1070D00021F76C2F81E190E0B5D1DFCF853031F41D
:1070E00021303105D1F6C093B206D7CF863031F4C6
:1070F0002130310591F6C093B506CFCF8730E1F44A
:107100002130310551F4CF3F19F41092B306C5CFA9
:10711000CC2319F2C093B306C0CF2230310509F059
:10712000BCCFCF3F19F41092B406B7CFCC2309F4EB
:10713000B4CFC093B406B1CF8130C9F42330310548
:1071400019F4C093DC02A9CF8C2F90E022303105D6
:1071500029F49093F5048093F4049FCF982F882707
:107160002091F4043091F504822B932BF2CF8330DD
:1071700009F093CFE5E9F5E0E21BF30BC0838DCF77
:1071800010920505CC2301F1C13009F58DE0EBE447
:10719000F5E0A7EFB4E001900D928A95E1F78091B8
:1071A00061058093F6048DE0D2DEE6EFF4E024E0A2
:1071B00035E08191909103058927809303052E176F
:1071C0003F07B9F78093F3048C2FCF910895C23015
:1071D00089F4809161058093F604EDE9F6E0A7EF6C
:1071E000B4E081918D9336E0E93AF307D1F78DE071
:1071F000AEDE5CCFC33039F588B18F7388B985E0D6
:107200008A95F1F7000088B1806C88B995E09A956D
:10721000F1F7000088B18F7388B935E03A95F1F73E
:10722000000080914B0580FD479A80914B0581FDC0
:10723000469A80E18A95F1F788B1806C88B987B168
:10724000806C87B933CFC43049F4E091BB06F0912C
:10725000BC0602A0F3A1E02D099528CF8091F3048C
:10726000C93009F4C1C0C13179F46091F40470915E
:10727000F504E0919A06F0919B060084F185E02DDB
:107280008091DC02099512CFC43161F46091F4045D
:107290007091F504E0919A06F0919B060284F385C3
:1072A000E02DEECFCA3159F4E0919A06F0919B0699
:1072B0000084F185E02D6AE070E08FEFE3CFCB3101
:1072C00041F4E0919A06F0919B060284F385E02D4B
:1072D000F2CFCC3151F483E090E090930705809396
:1072E000060581E080930505E1CEC03241F481E0DE
:1072F00090E0909307058093060582E0F3CFC132BA
:10730000C9F5809161058093F6042091B2068091C1
:10731000AA0638E0839FC00111244091A90630E1FC
:10732000439FA0011124842B90915B05892B4091F0
:10733000AC0690E2499FA0011124842B4091AB063A
:1073400030E4439FA0011124842B40915F0590E815
:10735000499FA0011124842B922F9160990F892BB2
:10736000226094E0299F90011124822B8093F704DE
:1073700082E03ECFC23241F487E190E0909307056E
:107380008093060583E0AECFC33241F481E090E004
:10739000909307058093060584E0A4CFC43241F49E
:1073A00081E090E0909307058093060585E09ACFF1
:1073B000C53241F481E090E0909307058093060583
:1073C00086E090CFC63241F482E090E090930705CA
:1073D0008093060587E086CF81EFCF3F29F4C093E5
:1073E000F60481E0B4DDF0CE8093F60481E000CFB6
:1073F00088ED92E00895A29FB001B39FC001A39FC2
:10740000700D811D1124911DB29F700D811D1124DD
:10741000911D0895FB01DC0102C001900D924150C5
:107420005040D8F70895DC0101C06D9341505040A1
:10743000E0F70895F999FECF92BD81BDF89A99279A
:1074400080B50895262FF999FECF92BD81BDF89A97
:10745000019700B4021639F01FBA20BD0FB6F89498
:0C746000FA9AF99A0FBE0895F894FFCF35
:10746C00A809E90965091B09D408CC083200010CEC
:10747C0004000000000000000200100A00010000DF
:10748C0000000002000000010200000E00010000DC
:10749C000000000000002001010020090100000094
:1074AC00C20C3E0D460C1C0C380C2A0CC10F0B0FD9
:1074BC006628090FEE0E080FD60F50106628F30F32
:1074CC00D70FF20F05D0109411CE10A313CF10CFFD
:1074DC001000F001B913F915B813CD14D413D71348
:1074EC00042B002A00290004250024002300022973
:1074FC000010032B002A002900012B002A00290070
:10750C0002290004022B002A002900202B002A004B
:10751C00290010230002012B002A002900082B004F
:10752C002A00290004290002012B002A002900014D
:10753C002B002A002900022900046C19B5196A19BC
:10754C008C196B196B19BA1ACF1BB81A2A1BB91ADA
:10755C00B91A4A1DE41D481D0E21491D491D0880FC
:10756C000088C000C8FF0048FF3F40FF80C0FFBF3D
:10757C00C1FFFF41BFFF0180FF813FFF8500FF0579
:10758C0000BF04008084003F8C00000C3F02008090
:10759C0080017D00B521D922B3212022B421B42150
:1075AC00019E2529267C25A6267D257D250A277961
:1075BC0027C9261627CA26CA265229D128E028B957
:1075CC0028EF286D2F2D290129D92E002A034700D9
:1075DC0061006D00650072002D00500072006F009C
:1075EC00200041006400760061006E0063006500BD
:1075FC0064002E0030000000120100020000004068
:10760C00D016040D00020102000101AE31B6317634
:10761C0037C6360D321F32313200364D327932C810
:10762C0031C93245332834E2358334C2346537618D
:10763C00376B36A231A931FFE8370438FF02010855
:10764C000480402001042420280818101400000095
:0A765C008080808080808080FF0025
:00000001FF
